:1065CD0001190000090101240200000301FA040071
:1065DD00FA0500030A0A5A0B001E0C00FA0D0003FF
:1065ED000E00030F0164100096120132130AFA1403
:1065FD00010215000217010A1801FA1905321A01D4
:10660D000A1B01FA1C05321FFFFF20FFFF23011E8D
:10661D002400642A00FA2B00FA2C50782D003D2E10
:10662D0000462F001E3000643250783432FA3501A6
:10663D0064360164370150380A643C00643E003C06
:10664D003F000140FFFF411450420A5A430AC8441B
:10665D0005324500B44600FA4701484802034C0094
:10666D00FA4EFFFF500808510596520A32530B4659
:10667D00540A96560202570546580002590A465AC0
:10668D0032FA5B010A5C0A325E000A5F00FE61FFAE
:10669D00FF6402106600026701016A0A3C6B00008C
:1066AD006C32967300007400007801327901327EED
:1066BD0000FE7FFFFF80FFFF8100008400FE85004C
:1066CD00AF8600018700FA8901078A000099000052
:1066DD009D0A969E00019FFFFFFAFAFA0065006F72
:1066ED0000790083008D009700A100AC00B600C0BA
:1066FD0000CA00D400DE00E800F2005B0063006A0F
:10670D000072007A008200890091009900A100A812
:10671D0000B000B800BF00C700CF00D600DF00E614
:10672D0000EE00F600400046004C00520059005F9C
:10673D000065006B00710077007D00830089008F7C
:10674D000095009C00A200A800AE00B400BA00C0E5
:10675D0000C600CC00D200D900DF00E500EB00F14F
:1035E7009007D0E0FEA3E0FF9065CF1268A6E493B2
:1035F700F5999065CDE493FC740193FDEFB505074C
:10360700EEB50403754D009007D012688D2285F939
:103617007285FA737E017F00E57312687FE5722F6A
:10362700FF50010E8E598F5A90001BE0FCA3E0FD5E
:10363700EF2DFDEE3CFC8C5B8D5C2275A71085F9A8
:103647007285FA737E017F00E57312687FE5722F3A
:10365700FF50010E8E598F5A90001BE0FCA3E0FD2E
:10366700EF2DFDEE3CFC8C5B8D5C22E55CF5FBE50C
:103677005BF5FCD29322E55CF5E9E55BF5EAD294CC
:1036870022E55CF5EBE55BF5ECD29122E55CF5ED27
:10369700E55BF5EED29222E55CF5FBE55BF5FCD246
:1036A7008722E55CF5E9E55BF5EAD29022E55CF572
:1036B700EBE55BF5ECE5B54410F5B522E55CF5ED1A
:1036C700E55BF5EEE5B54420F5B522AE59AF5A7482
:1036D7000A8E048F05FF12686F8C5B8D5CAE59AF45
:1036E7005A740A8E048F05FF12689A8C598D5AE511
:1036F7005A45596013740AC3955AFFE49559FE8ECB
:10370700598F5A785B1268D3E572A85BB80015D356
:10371700955C4010E572C3955CFFE4955BFE8E5B9C
:103727008F5C8010E5722424C3955CFFE4955BFEF3
:103737008E5B8F5CAE5BAF5C74236F4E6006742448
:103747006F4E701AAE5BAF5C74236F4E7005757267
:10375700018003757202755C22755B0080037572C8
:1037670000229000A0E0B40104C20D8002D20D90A7
:1037770000A1E0B40104C20E8002D20E9000DEE088
:1037870075F0E1A4FFAEF0740A8E048F05FF12688E
:103797006F9007C6ECF0A3EDF0A20A401674038CF5
:1037A700068D0712687F74011200399007C4EEF086
:1037B700A3EFF07E017F0090009CE012687F9000ED
:1037C700DFE08E048F05FF12686F740AFF12686FBF
:1037D7008D5F9000E8E075F0E1A4FFAEF0740A8E0B
:1037E700048F05FF12686F9007CAECF0A3EDF09005
:1037F70000EAE060139000EAE0F5F0741684FF7EBB
:1038070000EF9007D4F0800674649007D4F090001E
:10381700E0E0900084F090012AE090006EF09000C4
:10382700B9E0900070F09000E2E0900071F0900035
:103837008EE0900072F0900114E0900077F074E34E
:10384700900083F09000C9E0B40B0874E390008304
:10385700F0805A9000C9E0B419129000DFE090663A
:10386700D412008CE493900083F080419000C9E06B
:10387700B41E129000DFE09066F212008CE4939081
:103887000083F080289000C9E0B428129000DFE0A0
:1038970090671C12008CE493900083F0800F9000D7
:1038A700C9E0B446089000C0E0900083F09000871C
:1038B700E0FE9000C6E0B50633900088E0FE900079
:1038C700F2E0B50627900089E0FE9000E4E0B50637
:1038D7001B90008BE0FE900099E0B5060F90008AE0
:1038E700E0FE9000D4E06E7003023ACE9000D4E080
:1038F700640360069000F2E060087403900115F01D
:1039070080067407900115F09000F2E0B402089069
:1039170000D4E064036002800674009000F2F09027
:103927000099E0B4020674009000E4F0900099E07A
:10393700B4030674009000F1F09000E4E0D3940122
:10394700402774009000AEF0741B900117F07400CC
:103957009006D6F074009006D7F09000C6E0B40247
:103967000674019000C6F080339000C6E0B4021AD6
:10397700741B9000AEF07400900117F0740090066D
:10398700D6F074009006D7F0801274009000AEF065
:103997007400900117F0741B9006D6F09000D4E0E5
:1039A700B403089000F2E06402600280067400909D
:1039B70000F2F09000F2E0B401089000D4E0640354
:1039C70060028026741C900118F074009000ADF01E
:1039D70074009006DAF074009006DBF09000C6E001
:1039E700600674009000C6F080329000C6E0601A4E
:1039F700741C9000ADF07400900118F074009006EC
:103A0700DAF074009006DBF080127400900118F071
:103A170074009000ADF0741C9006DAF09000D4E0CA
:103A2700B402069000F2E06002801A74059006DE88
:103A3700F074069006E2F074079006E6F0740890BA
:103A470006ECF0803074009006DEF074009006DF1C
:103A5700F074009006E2F074009006E3F0740090B2
:103A670006E6F074009006E7F074009006EAF0743A
:103A7700009006EBF0D2289000C6E0900087F09007
:103A870000F2E0900088F09000E4E0900089F09068
:103A970000D4E090008AF0900099E090008BF090BD
:103AA7000099E090006FF09000D4E0900073F090E0
:103AB70000F2E0900074F09000C6E0900075F0907E
:103AC70000E4E0900076F09000FCE0B4011790006D
:103AD70027740FF0A374FFF0900029E4F0A3F074AB
:103AE700029000FCF09000FCE0B40341900029E054
:103AF700FEA3E0FF900027E0FCA3E0FD1268CB7473
:103B07001012687F7408120039EF900080F0EF7090
:103B17000674FF900080F074009000FCF09000287D
:103B2700E0900081F0900027E0900082F090008DF7
:103B3700E090004BF090004BE0240990004CF0908F
:103B4700004BE0241290004DF090004BE0241B90B6
:103B5700004EF090004CE0D39424400B90004CE0D2
:103B6700C3942490004CF090004DE0D39424400B74
:103B770090004DE0C3942490004DF090004EE0D3A8
:103B87009424400B90004EE0C3942490004EF09094
:103B97000053E4F090004BE06423600790004BE093
:103BA700B4242090004BE0B423067402900053F035
:103BB70090004BE0B424069000537401F090004B42
:103BC7007401F0900054E4F090004CE06423600727
:103BD70090004CE0B4242090004CE0B4230674021B
:103BE700900054F090004CE0B42406900054740107
:103BF700F090004C7401F0900055E4F090004DE017
:103C07006423600790004DE0B4242090004DE0B499
:103C170023067402900055F090004DE0B4240690FE
:103C270000557401F090004D7401F0900056E4F0D7
:103C370090004EE06423600790004EE0B42420908B
:103C4700004EE0B423067402900056F090004EE058
:103C5700B424069000567401F090004E7401F09061
:103C6700008DE0FE9000F0E02E900058F090005894
:103C7700E064126007900058E0B42406900058E012
:103C870004F0900058E064116007900058E0B423F6
:103C970006900058E014F0900058E0D39424400BAD
:103CA700900058E0C39424900058F0900058E0D357
:103CB7009412400D900058E0C39412900059F08080
:103CC7000A900058E02412900059F07550129000A5
:103CD700D3E090004FF090004FE075F00984AFF00B
:103CE7007E00EF4E700690004FE004F090004FE02A
:103CF7000475F00984AFF07E00EF4E700690004F18
:103D0700E014F090004FE0B4490690004F7401F0C2
:103D170090004FE0D39424400F90004FE0C39424C9
:103D270090004FF0D2238002C22390004FE0240975
:103D3700900050F090004FE02412900051F0900056
:103D47004FE0241B900052F0900050E0D3942440A1
:103D57000B900050E0C39424900050F0900051E085
:103D6700D39424400B900051E0C39424900051F069
:103D7700900052E0D39424400B900052E0C3942467
:103D8700900052F022C293C294C291C292C287C2DB
:103D970090E5B554EFF5B5E5B554DFF5B5C296C274
:103DA70095C2A0C297C2A2C2A1E5B554BFF5B5E5B9
:103DB700B5547FF5B5E5B554FBF5B5C20F755D464E
:103DC7009000D6E07005756C028003756C0375541E
:103DD7000075530090001074FFF0A374DCF0C21656
:103DE700C218C21AC21C74C890003BF074C8900075
:103DF7003FF074C8900043F074C8900047F07552C4
:103E070000755100C20A754600E56EB40903756E68
:103E17000075620090001DE4F0A3F0756F10C212E8
:103E2700C213C214C2159007C6E0FEA3E0FF7403D5
:103E370012687F74011200399007C4EEF0A3EFF007
:103E4700C202755600755500900014E4F0A3F0C245
:103E570029755800755700900098E075F032A4FD59
:103E6700ACF0900025ECF0A3EDF0C2392285F97291
:103E770085FA737E017F00E57312687FE5722FFF75
:103E870050010E8E598F5AAC5BAD5CEF2DFDEE3CA9
:103E9700FC8C5B8D5C12367212367D1236881236B8
:103EA700939000D4E0B4032C75A71085F97285FAB6
:103EB700737E017F00E57312687FE5722FFF500163
:103EC7000E8E598F5A12369E1236A91236B41236F2
:103ED700C375A7002275A71085F97285FA737E014D
:103EE7007F00E57312687FE5722FFF50010E8E5930
:103EF7008F5A7E017F76900111E012687FAC59AD31
:103F07005AED2FFFEC3EFE8E5B8F5CE55CF5FDE521
:103F17005BF5FE900084E4F075A700741290005BD7
:103F2700F02285F97285FA737E017F00E5731268C6
:103F37007FE5722FFF50010E8E598F5A9007C6E00A
:103F4700FCA3E0FDEF2DFDEE3CFC8C5B8D5CE55C9E
:103F5700F5FDE55BF5FE220563229000D4E06403DE
:103F670060079000F2E0B4021EA2D8B34002C293E9
:103F7700A2D9B34002C294A2DAB34002C291A2DB33
:103F8700B34002C2928044A2D8B3400AC2939000C1
:103F9700F2E06002C287A2D9B3400AC2949000F24D
:103FA700E06002C290A2DAB3400EC2919000F2E044
:103FB7006006E5B554EFF5B5A2DBB3400EC29290AB
:103FC70000F2E06006E5B554DFF5B5A2DCB34008C2
:103FD700C296C295C2A0C29775D8402285A77175AF
:103FE700A7109000D4E0640360079000F2E0B402E9
:103FF70024A2D8B34002C287A2D9B34002C290A27A
:10400700DAB34006E5B554EFF5B5A2DBB34006E5F4
:10401700B554DFF5B5A2DCB340089000E0E09000AE
:1040270084F075D8408571A722900047E493640611
:10403700600280FE74C89007CCF8E4F0E8A3F0753E
:10404700B50075840175A70075FFA0900057E4F0CF
:1040570075C91075A70F75A1C775A70075D9007524
:10406700CE0C75A70F75F1FE75F2FF75F30775F4A2
:104077007875A4BA75A5FF75A60775AE0075AFFF6D
:1040870075D48175D5FF75D6FF75D7FF75A70075F0
:10409700A20175A14775F80975D80075D90475DAB5
:1040A7000975DB0975DC0975DD0975DE0975D84009
:1040B70075A71075D80075D90475DA0975DB097508
:1040C700DC0975DD0975DE0975D84075A70075E649
:1040D7000875E71075BC0175BE0475BD6C75BE0724
:1040E70075BDA075BE0875BD0175BC0075BB18759B
:1040F700BC2075BA0875E88075D11375A70F75E1EF
:104107000575E20075C740123D8C7597007597805D
:10411700740A12685F7597C0E5975420700280F89B
:10412700758F0275A700D2AF75980075A90C75A792
:104137000F75AB4375ADFB75AC1E75A71075C91828
:1041470075CA0075CB0075C80475A7007589127507
:104157008E04758C00758A00C2A9D28C758D007586
:104167008B00D2ABD28E75EF0675D944C29974C84D
:10417700F5097508001200E375B5001204E37463CE
:104187009007CCF8E4F0E8A3F012036F74C8900727
:10419700CCF8E4F0E8A3F07464F5097508001200A0
:1041A700E390006FE0900099F0C220900099E0D36F
:1041B700940340067400900099F0900099E0906194
:1041C700DFF82828738028A2B44002D22080207507
:1041D700A70F75F30F75A700A2A34002D220800F87
:0F41E70075A70F75F31775A700A2A44002D22089
:0C61DF000241CC0241CE0241D60241E751
:1041F600A220B34066757208E572D3940E5020E58E
:10420600729007CCF8E4F0E8A3F012023E7464F56D
:10421600097508001200E37872740126F650D97405
:10422600029000D5F0900099E0D394034006740004
:10423600900099F0900099E09061EBF8282873803F
:104246001674009000FFF0800E74009000E4F08079
:074256000674009000F1F076
:0C61EB0002424502424702424F02425766
:10425D00D21F8064757201E572D394075020E57208
:10426D009007CCF8E4F0E8A3F012023E7464F5096F
:10427D007508001200E37872740126F650D97401A6
:10428D009000D5F0900099E0D3940340067400900F
:10429D000099F0900099E09061F7F8282873801646
:1042AD0074009000FFF0800E74009000E4F0800622
:0642BD0074009000F1F016
:0C61F7000242AB0242AD0242B50242BDC2
:1042C300C21F90006EE090012AF090006FE0900012
:1042D30099F0900070E09000B9F0900071E09000C8
:1042E300E2F0900072E090008EF0900073E0900096
:1042F300D4F0900074E09000F2F0900075E090002C
:10430300C6F0900076E09000E4F0900077E0900132
:1043130014F09000DFE07006740A9000DFF0900064
:10432300C0E0700674E39000C0F09000C6E0049013
:104333000087F0123769E5B54401F5B574069000BE
:104343005DF0740190005EF07403900060F07405FA
:10435300900061F0743E900062F07405900063F089
:104363007400900064F07400900069F07400900091
:104373006AF0740190006BF0740090006CF074FFAD
:1043830090006DF07433900163F07436900164F023
:10439300742D900165F07432900166F074209001E1
:1043A30067F0744C900168F07465900169F074785B
:1043B30090016AF0747590016BF0747390016CF066
:1043C300742090016DF0745690016EF07456900154
:1043D3006FF07454900170F07420900171F09000AC
:1043E300FBE0900080F09000B2E0900081F090003C
:1043F300B3E0900082F0A2B6B3920BA2B3B3920CD7
:10440300A2A4B39226A2A3B3922790007CE4F075F2
:104413006E00743A90078CF074FD90078DF0900055
:104423007DE4F09007C6E0FEA3E0FF740312687F0B
:1044330074011200399007C4EEF0A3EFF0756D011B
:1044430090005BE4F0C225756200C210D211C20273
:10445300757000C22BD203C22CD204C22DD205C266
:104463002ED206C22FD207C230D208C231D209C21D
:1044730021C222C223C224C22812009E755E007587
:104483006A0075600075643275650075660075674E
:104493000075680075690090001DE4F0A3F0756B6A
:1044A30000D2B2D2A4D2B0D2B1D2A3D2A7D2A6D2D2
:1044B300A5D2B7900098E0D394FA400674FA90001E
:1044C30098F07E017F00900082E012687F90008167
:1044D300E02FFF50010E900027EEF0A3EFF0EFD393
:1044E30094FFEE940F4007900027E4F0A3F09000B0
:1044F30080E0700674FF900080F074009000BFF0BD
:104503009000D5E0D39402400674019000D5F0905A
:1045130000D6E07005756C028003756C039000D7BC
:10452300E0D39401400674009000D7F09000DDE0E2
:10453300C3940A5006740A9000DDF09000E7E0701F
:104543000674019000E7F09000E7E0B4FF0674FE04
:104553009000E7F09000EEE0D394FE400674FE90E6
:1045630000EEF0900114E0D3940240067401900130
:1045730014F090012AE0D394014006740190012ABB
:10458300F074019000F4F074019000F5F074009061
:1045930000FCF07419900119F0741A90011AF07468
:1045A3002A90011BF0740090011CF074299006D22C
:1045B300F0D29C9000C7E0D39404400674049000AA
:1045C300C7F09000F9E0D39404400674049000F916
:1045D300F0E56FD394104003756F109006D3E0D3CA
:1045E300940C400674009006D3F09006D7E0D39461
:1045F3000C400674009006D7F09006DBE0D3940CD1
:10460300400674009006DBF09006DFE0D3940C4084
:104613000674009006DFF09006E3E0D3940C4006A6
:1046230074009006E3F09006E7E0D3940C40067420
:10463300009006E7F09006EBE0D3940C400674007C
:104643009006EBF0D2EC75CF01A298B34005C29867
:10465300120616E54D6006A299B3B340028005C267
:1046630099120AB4E54E64016005E54EB404028074
:10467300D5C28E7E107F00E56312687FE58D75F0ED
:1046830010A4FDACF0EF2DFDEE3CFCE58B75F010B6
:1046930084FF7E00ED2FFFEC3EFE8E538F54D28EAF
:1046A3009000B9E060099000B9E0C3943D400280F6
:1046B3005C90001F12688D90001FE0FEA3E0FF9046
:1046C3000021E0FCA3E0FDEFB50542EEB5043EB2E8
:1046D3001EA20AB3401975E700A21EB34008E5B550
:1046E3004404F5B58006E5B554FBF5B575E71090C0
:1046F3000021E0FEA3E0FF900023E0FCA3E0FDEF38
:104703002DFDEE3CFC900021ECF0A3EDF09000C6F3
:10471300E060099000C6E0C3940340030247C3125C
:1047230029C0A20AB3500990007CE0C3941F400241
:1047330080069000B0E0F545E54575F005A4FFAEB1
:10474300F09007CEEEF0A3EFF090009DE0C39560EC
:104753004007E55EC3955F50079007CEE4F0A3F0F2
:1047630075E700AE2EAF2F9007CEE0FCA3E0FDEF80
:10477300D39DEE9C4020E5B5547FF5B59000C6E08F
:10478300B402099000E4E0C3940240028006E5B558
:104793004440F5B5802790007CE0C3942E501EE57D
:1047A300B54480F5B59000C6E0B402099000E4E09A
:1047B300C3940240028006E5B554BFF5B575E71012
:1047C3009000C6E0B4032A122ADB75E700AE2EAFD1
:1047D3002F9007CEE0FCA3E0FDEFD39DEE9C4008B5
:1047E300E5B54480F5B58006E5B5547FF5B575E7C5
:1047F300109000A1E06009A2B3300C01B3B34002F2
:104803008039A2B3300C01B34031A2B3300E01B3EF
:10481300401C9000D4E0B40306A221B3B34002804D
:1048230006740490005BF0D221A20EB3920CA20E88
:10483300B330B301B34004A20E920CA2B6300B0105
:10484300B35003024EEFA2B6300B01B35003024E36
:10485300EFA2B6300D01B35003024D09756D009000
:1048630000B9E0B43D1975E700A20DB34008E5B502
:1048730054FBF5B58006E5B54404F5B575E71005B9
:104883005DA20FB3B35013AE53AF54900010E0FCCE
:10489300A3E0FDEDC39FEC9E40030249E6E56CB443
:1048A300032EA229B34022E55DB42303756C01E511
:1048B3005DC39423500690005B7401F0E55DD394CF
:1048C300234006740290005BF0755D01D229805E7F
:1048D300E56CB40206756C01755D23E55DB42305D3
:1048E300755D01804990005BE07034E55DC39423FE
:1048F300500690005B7401F0E55DD3942340067489
:104903000290005BF0E55DC394235002D225E55D80
:10491300D394234002D225C296C295C2A0C29790D7
:1049230000D6E0B40105123D8C8003755D01AE55E0
:10493300AF56AC53AD54EF2DFDEE3CFC74028C0628
:104943008D071200398E558F569000B9E06009909B
:1049530000B9E0C3943D4002804390001FE0FEA3F2
:10496300E0FF9000B9E08E048F05FF12686F7401B9
:104973008C068D07120039900023EEF0A3EFF09020
:104983000023E0F8A3E0900021C8F0A3C8F0900052
:104993001FE4F0A3F0C21EE5B554FBF5B5A2A4B322
:1049A3004002C226A2A3B34002C227A225B34002FB
:1049B300C225A221B34006A22392228002B22290F2
:1049C30000A1E06012E56C700EA221B35009A2228F
:1049D300302301B3B340028006740590005BF0C23C
:1049E30021803AAE55AF56AC53AD54EF2DFDEE3C9E
:1049F300FC74018C068D071200398E558F56E56CB9
:104A0300C39402500DAC53AD547488C39D74139C6E
:104A130040028009123D8C740690005BF0E55DB4A2
:104A23002312740390005BF0D2259000D6E0B4010A
:104A330003123D8CAE57AF58AC53AD54EF2DFDEE82
:104A43003CFC8C578D58AE53AF54EFD39DEE9C4036
:104A530011900017E0FAA3E0FBEBC394E8EA940398
:104A63004002800690001712688D900014E0FEA3A8
:104A7300E0FFAC53AD54EF2DFDEE3CFC900014EC85
:104A8300F0A3EDF09000D6E0B40118AE53AF547428
:104A93000512687F7401120039900010EEF0A3EF45
:104AA300F08011AE53AF54740212687F900010EE81
:104AB300F0A3EFF0C28E758D00758B0075630075E2
:104AC3005401755300D28EE55D240875F00984AF57
:104AD300F07E00EF4E7075900014E0F8A3E09000B4
:104AE30012C8F0A3C8F0900012E0FEA3E0FFEF4E5F
:104AF300600B7C817D5512676D8E518F529000142F
:104B0300E4F0A3F0AE51AF527428BE00039F5010DF
:104B1300E5622FFF50010E74011200398E518F523E
:104B23008552629000DDE0A851B8000DD395524044
:104B330008E55290005AF080099000DDE0149000DF
:104B43005AF0E56C60067552007551009000D4E090
:104B5300B4030890004FE0655D6002800BA222B3AE
:104B63004004D2248002B224E55D640B6005E55D58
:104B7300B41D099000C6E0600312202B900058E09A
:104B8300655D6007900059E0B55D03756E00A21086
:104B9300B35006A20FB3B34003024C44900092E01B
:104BA300B40173900114E0B40214120C5590008503
:104BB300E075F0BEA4FFAEF08E5B8F5C8056E566B9
:104BC30075F00A84FF7E0090058C1268A6E0F55A02
:104BD300755900AE59AF5A9000B7E012687F7464FC
:104BE3008E048F05FF12686F8C5B8D5CE55C900013
:104BF30016F0AE59AF5A900090E012687F74648E3D
:104C0300048F05FF12686F74BE8C068D0712687FD0
:104C13008E5B8F5C8017900090E075F0BEA4FFAEB2
:104C2300F08E5B8F5C9000B7E0900016F0E560C3F8
:104C330094CC5006900090E070028003123E74D230
:104C430010E56CB40106E55D640B60028009756FC5
:104C53000190005C7401F0E56C6003024D04900068
:104C6300D9E0600D900084E0A851B8000695524049
:104C73000280489000D9E0B4022790004BE0655DC4
:104C8300601790004CE0655D600F90004DE0655D3E
:104C9300600790004EE0B55D03756F03756B008090
:104CA3000CC200756B0090001DE4F0A3F09000842B
:104CB300E06006740990005BF0804690004BE0B51D
:104CC3005D0B756F0190005C7401F0803490004CB3
:104CD300E0B55D0B756F01740290005CF08022906B
:104CE300004DE0B55D0B756F01740390005CF080BF
:104CF3001090004EE0B55D09756F01740490005C7F
:104D0300F0A20DB3920BA20DB330B601B350030260
:104D13004EEF756D019000B9E0B43D1975E700A23F
:104D23000DB34008E5B54404F5B58006E5B554FB7D
:104D3300F5B575E710E5B54401F5B5741F90007C32
:104D4300F0A20D920BE55DD3944A4014D20FE55DBA
:104D5300D3946D400B740490005BF0D225755D46CF
:104D63009000E1E0B40107E569C3941440028009AF
:104D7300123D8C741390005BF0A22B300301B350EF
:104D83001D75E700A22BB34008E5B54408F5B580CF
:104D930006E5B554F7F5B575E710A22B9203A22CDF
:104DA300300401B3501D75E700A22CB34008E5B5EC
:104DB3004440F5B58006E5B554BFF5B575E710A2D7
:104DC3002C9204A22D300501B3501D75E700A22DCE
:104DD300B34008E5B54480F5B58006E5B5547FF5E5
:104DE300B575E710A22D9205A22E300601B3500F20
:104DF300A22EB34004D2878002C287A22E9206A2BB
:104E03002F300701B3500FA22FB34004D29080027A
:104E1300C290A22F9207A230300801B3501D75E74C
:104E230000A230B34008E5B54410F5B58006E5B5FA
:104E330054EFF5B575E710A2309208A2313009019D
:104E4300B3501D75E700A231B34008E5B54420F522
:104E5300B58006E5B554DFF5B575E710A2319209C3
:104E630075E70090010FE0A851B80005D3955250A3
:104E73000D90010EE0A851B800049552500280082D
:104E8300E5B54402F5B58017900110E0D395604075
:104E930008E5B54402F5B58006E5B554FDF5B575ED
:104EA300E710E569C394415009740E90005BF0125A
:104EB3003D8C900063E0FE90005FE0C39E4009904C
:104EC300005FE0D39406400974FB90005BF0123D51
:104ED3008C900068E06015900068E0FE900062E04E
:104EE3006E600974FE90005BF0123D8CA225B34006
:104EF30008C296C295C2A0C297900111E0600CAEA1
:104F030051AF527414BE00059F4002803790009940
:104F1300E0906203F8282873802A8028A2A3B35064
:104F230005A227B340028005123EDCD2278015A2DA
:104F3300A4B35005A226B340028005123EDCD2265C
:044F43008002800068
:10620300024F1B024F1D024F1F024F32024F450226
:026213004F47F3
:104F4700A212B3B3500890004FE0655D60030250B2
:104F57001CA201B35006A200B3B340030250149041
:104F670000D4E0B4036EA20AB34038A224B34008C9
:104F7700123615123672800912364212369E75A7FE
:104F8700009000F2E0B4011975E700A202B34008EF
:104F9700E5B54480F5B58006E5B5547FF5B575E709
:104FA70010802F12361512367212364212369E753F
:104FB700A7009000F2E0B4011975E700A202B34020
:104FC70008E5B54480F5B58006E5B5547FF5B575B8
:104FD700E71080399000F2E0C39402500F123615A3
:104FE700123672A202B34002D287802112361512FE
:104FF7003672123642AE59AF5AAC2CAD2DEF2DFD9D
:10500700EE3CFC8C5B8D5C12369E75A700C212D2FB
:1050170013D214D215A213B3B35008900050E06511
:105027005D60030250F1A201B35006A200B3B34082
:10503700030250E99000D4E0B4036EA20AB34038EB
:10504700A224B3400812361512367D800912364263
:105057001236A975A7009000F2E0B4011975E700B0
:10506700A202B34008E5B54480F5B58006E5B5541E
:105077007FF5B575E710802F12361512367D12367B
:10508700421236A975A7009000F2E0B4011975E73E
:1050970000A202B34008E5B54480F5B58006E5B542
:1050A700547FF5B575E71080399000F2E0C394029C
:1050B700500F12361512367DA202B34002D29080ED
:1050C7002112361512367D123642AE59AF5AAC2C24
:1050D700AD2DEF2DFDEE3CFC8C5B8D5C1236A9757A
:1050E700A700D212C213D214D215A214B3B3500818
:1050F700900051E0655D60030251CAA201B35006FA
:10510700A200B3B340030251C29000D4E0B4036ECF
:10511700A20AB34038A224B34008123615123688C3
:1051270080091236421236B475A7009000F2E0B437
:10513700011975E700A202B34008E5B54480F5B54B
:105147008006E5B5547FF5B575E710802F12361543
:105157001236881236421236B475A7009000F2E074
:10516700B4011975E700A202B34008E5B54480F51C
:10517700B58006E5B5547FF5B575E710803D90001D
:10518700F2E0C394025013123615123688A202B306
:105197004006E5B54410F5B580211236151236885C
:1051A700123642AE59AF5AAC2CAD2DEF2DFDEE3C69
:1051B700FC8C5B8D5C1236B475A700D212D213C279
:1051C70014D215A215B3B35008900052E0655D6084
:1051D700030252A3A201B35006A200B3B3400302D5
:1051E700529B9000D4E0B4036EA20AB34038A224C5
:1051F700B34008123615123693800912364212361A
:10520700C375A7009000F2E0B4011975E700A20288
:10521700B34008E5B54480F5B58006E5B5547FF59C
:10522700B575E710802F12361512369312364212D3
:1052370036C375A7009000F2E0B4011975E700A224
:1052470002B34008E5B54480F5B58006E5B5547F5F
:10525700F5B575E710803D9000F2E0C39402501356
:10526700123615123693A202B34006E5B54420F56F
:10527700B58021123615123693123642AE59AF5AFF
:10528700AC2CAD2DEF2DFDEE3CFC8C5B8D5C12360E
:10529700C375A700D212D213D214C215E56F90625C
:0C52A70015F82828730258569000F9E012
:066215000252AC0252AF80
:1052B300906248F8282873121B078012121B07807C
:0E52C3000D121B918008121C3D8003121C3D31
:0F6248000252BA0252BF0252C40252C90252CECF
:1052D100756F02025856121D69121E80A239B34021
:1052E100229000BBE0F56B90008CE0256BFE9000F6
:1052F1005AE075F01E84FC7F00EE2CF5347410909A
:10530100005BF09007C4E0FEA3E0FF740A12687F1F
:10531100900012E0FCA3E0FD74098F02FF12686F98
:105321008D078C038E048A058B0612676D9007C862
:10533100EEF0A3EFF074F0BE00039F500B74F090F9
:1053410007C8F8E4F0E8A3F0E53470037534019080
:1053510007C8E0FEA3E0FFE5342FFF50010E9007E0
:0D536100C8EEF0A3EFF0756F0390005CE064
:03621B000252D755
:10536E00906257F82828738022A23A4003756F0A7C
:10537E008019A23A4003756F0B8010A23A40037554
:0B538E006F0C8007A23A4003756F0D02
:0F62570002537502537702538002538902539208
:105399000258569006D3E06003122114900112E0DE
:1053A900B40114900113E0A851B8000495525007B4
:1053B900E55EC3955F400280030254469000C7E052
:1053C900D39402403F90009BE02403A851B8000405
:1053D9009552500990009DE0D3956050028008D203
:1053E90001740890005BF090009BE0A851B800059B
:1053F900D39552500B90009DE02403C39560500251
:10540900C201803990009BE02403A851B80004959B
:10541900525007E55EC3955F40028008D2017408C7
:1054290090005BF090009BE0A851B80005D395521D
:105439005009E55F240FC3955E5002C2019000E157
:10544900E07007E569C3941440028002D201A20109
:105459004005756F04800A756F1090001DE4F0A374
:10546900F0A20AB34029E56675F00A84FF7E009030
:10547900058C1268A6E0C394695005122060800F5C
:105489009007C6E0F8A3E09007C4C8F0A3C8F002EB
:0654990058569000C7E028
:06621E0002539C02549B98
:10549F00906266F8282873120D3F8012120D3F801C
:0E54AF000D120EED8008120F9F8003120F9F4A
:0F6266000254A60254AB0254B00254B50254BA0B
:1054BD009006D7E060031221F0756F050258561261
:1054CD0010AB756F069006DBE060031222E09006CC
:1054DD00DFE060031223BC025856900016E0600610
:1054ED00A20AB3B34002801D900016E02529FFAE3D
:1054FD002850010E8E288F29E55DD3940950069012
:10550D000016E014F01212F1756F079006E3E060DB
:10551D00031224989006E7E0600312257402585692
:10552D00900114E0B40203120CCD12154E756F08E4
:10553D009006EBE0600312265002585612190AA28B
:10554D0012B35005A213B340028008D212D213D267
:10555D0014D215756F1002585602585690003DE042
:10556D00C394465008C296744690003DF090005387
:10557D00E0B4011DE534240AF5349007C8E0FEA31C
:10558D00E0FF740A2FFF50010E9007C8EEF0A3EF55
:10559D00F0900053E0B4021DE5342414F534900767
:1055AD00C8E0FEA3E0FF74142FFF50010E9007C852
:1055BD00EEF0A3EFF085345A75590090004BE0F5ED
:1055CD00721236D2E55C90003DF0900008E559F07E
:1055DD00A3E55AF0E57290003EF0C2179007C8E0BF
:1055ED00F559A3E0F55A90004BE0F5721236D2E56D
:1055FD005C90003BF0900000E559F0A3E55AF0E512
:10560D007290003CF0C216E56CB40105756F0B800D
:10561D0003756F03025856900041E0C3944650083D
:10562D00C2957446900041F0900054E0B4011DE520
:10563D0034240AF5349007C8E0FEA3E0FF740A2F66
:10564D00FF50010E9007C8EEF0A3EFF0900054E06C
:10565D00B4021DE5342414F5349007C8E0FEA3E030
:10566D00FF74142FFF50010E9007C8EEF0A3EFF05A
:10567D0085345A75590090004CE0F5721236D2E51A
:10568D005C900041F090000AE559F0A3E55AF0E571
:10569D0072900042F0C2199007C8E0F559A3E0F5E9
:1056AD005A90004CE0F5721236D2E55C90003FF056
:1056BD00900002E559F0A3E55AF0E572900040F034
:1056CD00C218E56CB40105756F0C8003756F03028C
:1056DD005856900045E0C394465008C2A0744690B9
:1056ED000045F0900055E0B4011DE534240AF53471
:1056FD009007C8E0FEA3E0FF740A2FFF50010E9043
:10570D0007C8EEF0A3EFF0900055E0B4021DE534AC
:10571D002414F5349007C8E0FEA3E0FF74142FFFA6
:10572D0050010E9007C8EEF0A3EFF085345A75596D
:10573D000090004DE0F5721236D2E55C900045F018
:10574D0090000CE559F0A3E55AF0E572900046F093
:10575D00C21B9007C8E0F559A3E0F55A90004DE043
:10576D00F5721236D2E55C900043F0900004E559D5
:10577D00F0A3E55AF0E572900044F0C21AE56CB45E
:10578D000105756F0D8003756F0302585690004922
:10579D00E0C394465008C2977446900049F09000BB
:1057AD0056E0B4011DE534240AF5349007C8E0FE37
:1057BD00A3E0FF740A2FFF50010E9007C8EEF0A36F
:1057CD00EFF0900056E0B4021DE5342414F534904A
:1057DD0007C8E0FEA3E0FF74142FFF50010E9007E1
:1057ED00C8EEF0A3EFF085345A75590090004EE0E5
:1057FD00F5721236D2E55C900049F090000EE55935
:10580D00F0A3E55AF0E57290004AF0C21D9007C86A
:10581D00E0F559A3E0F55A90004EE0F5721236D23C
:10582D00E55C900047F0900006E559F0A3E55AF0CD
:10583D00E572900048F0C21CE56CB40103756C0074
:09584D00756F03800480028000E5
:106224000254CC0254E702552D0255490255660228
:1062340055690256240256DF02579A0258520258F0
:046244005402585652
:1058560090003BE0B55D0280030258F8A216407244
:10586600900000E0FEA3E0FFEF4E6021AE55AF567C
:10587600900000E0FCA3E0FD120003740A8E048F82
:1058860005FF12686F900000ECF0A3EDF090003C6D
:10589600E0601A900000E0FEA3E0FFAC55AD56EFC5
:1058A6002DFDEE3CFC900000ECF0A3EDF090003CEA
:1058B600E0D39401401A900000E0FEA3E0FFAC554F
:1058C600AD56EF2DFDEE3CFC900000ECF0A3EDF0A4
:1058D600D216AE53AF54900000E0FCA3E0FDEFC338
:1058E6009DEE9C400D123F29D296C21674C89000B8
:1058F6003BF0A216B3B3500790003BE0B55D0280C3
:105906000D123F29D29674C890003BF0C216900043
:105916003DE0B55D0280030259B3A21740729000C4
:1059260008E0FEA3E0FFEF4E6021AE55AF569000B3
:1059360008E0FCA3E0FD120003740A8E048F05FF45
:1059460012686F900008ECF0A3EDF090003EE06066
:105956001A900008E0FEA3E0FFAC55AD56EF2DFD12
:10596600EE3CFC900008ECF0A3EDF090003EE0D396
:105976009401401A900008E0FEA3E0FFAC55AD5636
:10598600EF2DFDEE3CFC900008ECF0A3EDF0D217F5
:10599600AE53AF54900008E0FCA3E0FDEFC39DEECC
:1059A6009C400AC296744690003DF0C217A217B3F7
:1059B600B3500790003DE0B55D02800AC29674467A
:1059C60090003DF0C21790003FE0B55D02800302F3
:1059D6005A6EA2184072900002E0FEA3E0FFEF4E5E
:1059E6006021AE55AF56900002E0FCA3E0FD120028
:1059F60003740A8E048F05FF12686F900002ECF0A4
:105A0600A3EDF0900040E0601A900002E0FEA3E0F3
:105A1600FFAC55AD56EF2DFDEE3CFC900002ECF0D0
:105A2600A3EDF0900040E0D39401401A900002E00C
:105A3600FEA3E0FFAC55AD56EF2DFDEE3CFC90000D
:105A460002ECF0A3EDF0D218AE53AF54900002E092
:105A5600FCA3E0FDEFC39DEE9C400D123F29D295BD
:105A6600C21874C890003FF0A218B3B35007900054
:105A76003FE0B55D02800D123F29D29574C89000B3
:105A86003FF0C218900041E0B55D028003025B2939
:105A9600A219407290000AE0FEA3E0FFEF4E6021DB
:105AA600AE55AF5690000AE0FCA3E0FD1200037469
:105AB6000A8E048F05FF12686F90000AECF0A3EDC2
:105AC600F0900042E0601A90000AE0FEA3E0FFAC0E
:105AD60055AD56EF2DFDEE3CFC90000AECF0A3ED23
:105AE600F0900042E0D39401401A90000AE0FEA331
:105AF600E0FFAC55AD56EF2DFDEE3CFC90000AECF8
:105B0600F0A3EDF0D219AE53AF5490000AE0FCA317
:105B1600E0FDEFC39DEE9C400AC29574469000419D
:105B2600F0C219A219B3B35007900041E0B55D0267
:105B3600800AC2957446900041F0C219900043E075
:105B4600B55D028003025BE4A21A4072900004E095
:105B5600FEA3E0FFEF4E6021AE55AF56900004E085
:105B6600FCA3E0FD120003740A8E048F05FF126881
:105B76006F900004ECF0A3EDF0900044E0601A9002
:105B86000004E0FEA3E0FFAC55AD56EF2DFDEE3C64
:105B9600FC900004ECF0A3EDF0900044E0D39401F7
:105BA600401A900004E0FEA3E0FFAC55AD56EF2D81
:105BB600FDEE3CFC900004ECF0A3EDF0D21AAE53DF
:105BC600AF54900004E0FCA3E0FDEFC39DEE9C40C3
:105BD6000D123F29D2A0C21A74C8900043F0A21A2F
:105BE600B3B35007900043E0B55D02800D123F2924
:105BF600D2A074C8900043F0C21A900045E0B55D8B
:105C0600028003025C9FA21B407290000CE0FEA380
:105C1600E0FFEF4E6021AE55AF5690000CE0FCA3BE
:105C2600E0FD120003740A8E048F05FF12686F9060
:105C3600000CECF0A3EDF0900046E0601A90000C2A
:105C4600E0FEA3E0FFAC55AD56EF2DFDEE3CFC901B
:105C5600000CECF0A3EDF0900046E0D39401401A5E
:105C660090000CE0FEA3E0FFAC55AD56EF2DFDEE27
:105C76003CFC90000CECF0A3EDF0D21BAE53AF54FD
:105C860090000CE0FCA3E0FDEFC39DEE9C400AC231
:105C9600A07446900045F0C21BA21BB3B3500790F8
:105CA6000045E0B55D02800AC2A07446900045F04A
:105CB600C21B900047E0B55D028003025D5AA21C3C
:105CC6004072900006E0FEA3E0FFEF4E6021AE5565
:105CD600AF56900006E0FCA3E0FD120003740A8EA6
:105CE600048F05FF12686F900006ECF0A3EDF090AC
:105CF6000048E0601A900006E0FEA3E0FFAC55AD58
:105D060056EF2DFDEE3CFC900006ECF0A3EDF09076
:105D16000048E0D39401401A900006E0FEA3E0FF9D
:105D2600AC55AD56EF2DFDEE3CFC900006ECF0A315
:105D3600EDF0D21CAE53AF54900006E0FCA3E0FD9C
:105D4600EFC39DEE9C400D123F29D297C21C74C82A
:105D5600900047F0A21CB3B35007900047E0B55D32
:105D660002800D123F29D29774C8900047F0C21CDA
:105D7600900049E0B55D028003025E15A21D4072E7
:105D860090000EE0FEA3E0FFEF4E6021AE55AF5649
:105D960090000EE0FCA3E0FD120003740A8E048F4F
:105DA60005FF12686F90000EECF0A3EDF090004A2C
:105DB600E0601A90000EE0FEA3E0FFAC55AD56EF92
:105DC6002DFDEE3CFC90000EECF0A3EDF090004AA9
:105DD600E0D39401401A90000EE0FEA3E0FFAC551C
:105DE600AD56EF2DFDEE3CFC90000EECF0A3EDF071
:105DF600D21DAE53AF5490000EE0FCA3E0FDEFC3FE
:105E06009DEE9C400AC2977446900049F0C21DA2BE
:105E16001DB3B35007900049E0B55D02800AC297F2
:105E26007446900049F0C21D9000E4E0B40202807E
:105E360003025F5C90007EE0D39565506490007E1F
:105E4600E0F4042565FE9000E7E08E00F5F0E884B6
:105E5600FF7E008F72EFC39410500CEF8572F0A492
:105E6600FDACF08D7280037572FF90007EE0D395D5
:105E760072400B90007EE0C39572F57080037570DA
:105E860000900102E0D395704006900102E0F570A3
:105E9600900103E0C395705006900103E0F5708011
:105EA6007190007EE0C39565FE9000E7E08E00F5F8
:105EB600F0E884FF7E008F72EFC39410500CEF85DC
:105EC60072F0A4FDACF08D7280037572FF85725A74
:105ED60075590090007EE0255AFFAE5950010E8E8E
:105EE600598F5A74FFBE0009D39F4005855A7080AA
:105EF600037570FF900102E0D39570400690010291
:105F0600E0F570900103E0C395705006900103E040
:105F1600F570A20AB3B3500D90007FE0FE9000EF3B
:105F2600E0D39E5002800E740790005BF0E5B554F6
:105F3600BFF5B5802175A71075E700E5CDC395704F
:105F46004008E5B554BFF5B58006E5B54440F5B55E
:105F560075E71075A700900109E0A851B80005D3B0
:105F660095525016900108E0A851B8000D95524080
:105F76000990010AE0D395604002802175A710A21E
:105F86000AB3B35007E5CDC394BF40028004D2A242
:105F96008002C2A2A2A292A175A700801F75A710B7
:105FA600A20AB3B35007E5CDC3944040028004D2A1
:105FB600A28002C2A2A2A292A175A700E56EC39416
:105FC60009500AA2EDB34005C2ED122C7AAE53AFCA
:105FD600547498C39F743A9E400C90007DE0C3941D
:105FE6005A40030261DCA20FB34009123D8C7406CD
:105FF60090005BF0A220B34008E5B54404F5B580F7
:1060060006E5B554FBF5B5A211B3500EE560D39481
:10601600334007E560C394CC4002802FE5B54401C8
:10602600F5B5741F90007CF0900090E075F0BEA46A
:10603600FFAEF08E5B8F5C7402BE000AD39F4006F3
:10604600755C02755B00123E74D21190007DE0D340
:1060560094014007E560C3941A40028002C2119081
:1060660006D3E06003122114A22B300301B35017AC
:10607600A22BB34008E5B54408F5B58006E5B5544E
:10608600F7F5B5A22B92039006D7E060031221F034
:10609600A22C300401B35017A22CB34008E5B54436
:1060A60040F5B58006E5B554BFF5B5A22C9204902F
:1060B60006DBE060031222E0A22D300501B3501783
:1060C600A22DB34008E5B54480F5B58006E5B55484
:1060D6007FF5B5A22D92059006DFE060031223BC82
:1060E600A22E300601B3500FA22EB34004D28780F1
:1060F60002C287A22E92069006E3E060031224985D
:10610600A22F300701B3500FA22FB34004D29080C4
:1061160002C290A22F92079006E7E0600312257450
:10612600A230300801B35017A231B34008E5B54498
:1061360010F5B58006E5B554EFF5B5A23092089096
:1061460006EBE06003122650A231300901B3501766
:10615600A231B34008E5B54420F5B58006E5B5544F
:10616600DFF5B5A231920990007DE0C3945A501034
:10617600E56EB4090990007DE004F0756E00803B81
:10618600E56EB40903756E00755400755300758D80
:1061960000758B0075630090007CE0C3942E500858
:1061A60090007CE004F08006742E90007CF0900055
:1061B6007CE0B42E06E5B554FEF5B590007DE0D33F
:1061C60094014007E569C3944140028009740E902A
:0961D600005BF0123D8C02464909
:106275000000010001400160018001A001C001E0B2
:1062850002000300039603B603D603F404000500D9
:106295000512052405360548055A056C057E059049
:1062A50005A805C005DE0600061406280646066E86
:1062B50006AE00FF013F015F017F019F01BF01DFC6
:1062C50001FF02FF039503B503D503F303FF04FFA5
:1062D50005110523053505470559056B057D058F11
:1062E50005A705BF05DD05F1061306270645066D5D
:1062F50006AD06ED0FAA0FA50F9F0F9A0F940F8DF0
:106305000F870F800F780F710F680F600F570F4EB3
:106315000F450F3B0F300F250F1A0F0E0F020EF50D
:106325000EE80EDB0ECC0EBE0EAE0E9F0E8E0E7D53
:106335000E6C0E5A0E470E340E200E0C0DF70DE2A4
:106345000DCB0DB50D9D0D850D6D0D540D3A0D2023
:106355000D050CE90CCE0CB10C940C760C580C3ACE
:106365000C1B0BFB0BDB0BBB0B9A0B790B570B3584
:106375000B130AF10ACE0AAB0A870A640A400A1C03
:1063850009F809D409B0098C09670943091F08FBF5
:1063950008D608B2088E086A0846082307FF07DCF6
:1063A50007B9079607730751072F070D06EC06CAAD
:1063B50006AA068906690649062A060A05EC05CDD8
:1063C50005B0059205750558053C0520050504EA47
:1063D50004CF04B5049C04820469045104390422E1
:1063E500040B03F403DE03C803B2039D038903759D
:1063F5000361034D033B03280316030402F202E184
:1064050002D102C002B002A00291028202730265AB
:1064150002570249023C022F02220216020901FD1F
:1064250001F201E601DB01D001C601BB01B101A703
:10643500019D0194018B0182017901700168016060
:10644500015801500148014101390132012B012553
:10645500011E01180111010B010500FF00FA0FA62D
:106465000FA00F990F920F8B0F840F7C0F740F6B7A
:106475000F620F580F4E0F430F380F2C0F1F0F12BF
:106485000F050EF70EE80ED80EC80EB70EA50E9323
:106495000E800E6C0E580E420E2C0E150DFD0DE4E1
:1064A5000DCB0DB10D950D790D5D0D3F0D200D0138
:1064B5000CE10CC00C9E0C7C0C590C350C100BEA35
:1064C5000BC40B9E0B760B4F0B260AFD0AD40AAAAA
:1064D5000A800A550A2A09FF09D409A8097C095026
:1064E500092508F908CD08A10875084A081E07F30B
:1064F50007C8079D07730749072006F706CE06A6B6
:10650500067E06570630060A05E405BF059B057796
:1065150005540532051004EF04CE04AE048F047152
:1065250004530435041903FD03E203C703AD0394C3
:10653500037B0363034B0334031E030802F302DEEC
:1065450002CA02B602A30291027F026D025C024CEE
:10655500023C022C021D020E020001F201E401D7E9
:1065650001CA01BE01B101A6019A018F0185017A17
:1065750001700166015D0153014A01410139013193
:106585000129012101190112010B010400FD00F788
:1065950000F000EA00E400DE00D900D300CE00C917
:1065A50000C400BF00BA00B500B100AD00A800A44A
:1065B50000A0009C009900950091008E008A00873C
:0865C50000840081007E007BD0
:10009E007547009007D0E4F0A3F07531007530007D
:1000AE00754D00754E00C236D23774FE9007DAF8E1
:1000BE00E4F0E8A3F074FE9007DCF8E4F0E8A3F0B7
:1000CE00745A9007DEF0745A9007DFF0D238C22AC5
:1000DE00C23AC23522750B00750A00AE0AAF0BACE0
:1000EE0008AD09EDC39FEC9E401674FF12685F7554
:1000FE00CF01780B740126F6500418E436F650DB67
:10010E0022900057E0B4AA1C90078CE0B43C1590E6
:10011E0007CCE0FEA3E0FFEF4E6009741EBE0004A4
:10012E00D39F500302023D755C00755B0075F809A4
:10013E009007CCE0FEA3E0FF74076F4E6006740ECE
:10014E006F4E7006743A90078CF09007CCE0FEA3C9
:10015E00E0FF7408BE001ED39F401A7E017F0890F8
:10016E0007CCE0FCA3E0FD1DBDFF011C1200038EB9
:10017E00598F5A801F9007CCE0FEA3E0FF7408123F
:10018E0068C38F048E057E017F08CDCCCD1200038F
:10019E008E598F5AAE5BAF5C740CD39F74019E5018
:1001AE0003020238A2F9B3407EE55C455B7003752D
:1001BE00A382AE5BAF5C74016F4E700375A300AE8D
:1001CE005BAF5C74026F4E700D9007CDE075F00260
:1001DE00A4FDACF08DA3AE5BAF5C74036F4E7003E9
:1001EE0075A300AE5BAF5C7403BE00039F5013ACEF
:1001FE0059AD5AED2FFFEC3EFE9000881268A6E036
:10020E00F5A3AE5BAF5CEFB40B09EEB4010574144D
:10021E0012685FAE5BAF5CEFB40B07EEB401037513
:10022E00F80D785B1268D30201A2900057E4F02219
:10023E00755C00755B0075F8099007CCE0FEA3E0D5
:10024E00FF7408BE001ED39F401A7E017F089007E0
:10025E00CCE0FCA3E0FD1DBDFF011C1200038E5976
:10026E008F5A801F9007CCE0FEA3E0FF740812683F
:10027E00C38F048E057E017F08CDCCCD1200038E78
:10028E00598F5AAE5BAF5C7411D39F74019E5003AD
:10029E0002036EA2F9B3500302036BE55C455B707B
:1002AE000375A3D2AE5BAF5C74016F4E700375A382
:1002BE0000AE5BAF5C74026F4E700D9007CDE075B3
:1002CE00F002A4FDACF08DA3AE5BAF5C74036F4E79
:1002DE00700375A300AE5BAF5C74046F4E70037554
:1002EE00A300AE5BAF5C74056F4E700375A300AEDA
:1002FE005BAF5C74066F4E700375A300AE5BAF5CB4
:10030E0074076F4E700375A300AE5BAF5C74086F1D
:10031E004E700375A300AE5BAF5C7408BE00039F06
:10032E005016AC59AD5AED2FFFEC3EFE90008312E5
:10033E0068A6E5A3F075A300AE5BAF5CEFB4100941
:10034E00EEB40105741412685FAE5BAF5CEFB410CF
:10035E0007EEB4010375F80D785B1268D3020291B3
:10036E0022755C00755B0075F809AE5BAF5C7417A7
:10037E00BE0004D39F5003020447A2F9B3500302F8
:10038E000444E55C455B700375A3D2AE5BAF5C7451
:10039E00016F4E700375A300AE5BAF5C74026F4EBF
:1003AE00700D9007CDE075F002A4FDACF08DA3AEFC
:1003BE005BAF5C74036F4E700375A300AE5BAF5CF6
:1003CE0074046F4E700375A300AE5BAF5C74056F63
:1003DE004E700375A300AE5BAF5C74066F4E700378
:1003EE0075A300AE5BAF5C74076F4E700375A30010
:1003FE00AE5BAF5C74086F4E700375A300AE5BAF5F
:10040E005C7408BE00039F500C9000651268A6E550
:10041E00A3F075A300AE5BAF5C74166F4E700574DF
:10042E001412685FAE5BAF5C74166F4E700375F896
:10043E000D785B1268D302037822900057E0B4ABBC
:10044E000280030204E2755C00755B0075F809AE6C
:10045E005BAF5C7412BE007CD39F4078A2F9B340B0
:10046E0070E55C455B700375A382AE5BAF5C740197
:10047E006F4E700375A300AE5BAF5C74026F4E706F
:10048E000D9007CDE075F002A4FDACF08DA3AE5B30
:10049E00AF5C74036F4E700375A300AE5BAF5C74FC
:1004AE0003BE00039F500990006A1268A6E0F5A3F0
:1004BE00AE5BAF5C74116F4E7005741412685FAE54
:1004CE005BAF5C74116F4E700375F80D785B12683C
:1004DE00D302045D229007D7E4F074649007CCF841
:1004EE00E4F0E8A3F012036F74C89007CCF8E4F0C0
:1004FE00E8A3F0900071E0B4371A90006EE090001F
:10050E0065F090006FE0900066F0900070E0900053
:10051E0067F080469007D77401F074659007CCF8A9
:10052E00E4F0E8A3F012036F74C89007CCF8E4F07F
:10053E00E8A3F0900071E0B4371A90006EE09000DE
:10054E0065F090006FE0900066F0900070E0900013
:10055E0067F0800674029007D7F09007D8E4F07425
:10056E00669007CCF8E4F0E8A3F012036F74C8901D
:10057E0007CCF8E4F0E8A3F0900070E0B4371290E6
:10058E00006EE090005FF090006FE0900068F080E9
:10059E00769007D87401F074679007CCF8E4F0E811
:1005AE00A3F012036F74C89007CCF8E4F0E8A3F040
:1005BE00900070E0B4371290006EE090005FF09003
:1005CE00006FE0900068F0803E74029007D8F074DF
:1005DE00689007CCF8E4F0E8A3F012036F74C890AB
:1005EE0007CCF8E4F0E8A3F0900070E0B437129076
:1005FE00006EE090005FF090006FE0900068F08079
:10060E000674039007D8F022E54E64046006E5995F
:10061E0064FF6002802AA2364004D2368020E54E66
:10062E00600874E6254E90005BF0754E00E54D6057
:10063E000874F0254D90005BF0754D00C2368002B7
:10064E00C236E54E9033F8F8282873754E00E599BA
:10065E00B4FF03754D01E599B4FE03754D02E5999E
:10066E00B4FD03754D03E599B4FC03754D04E5998E
:10067E00B4FA03754D05E599B4FB06754E01123DAE
:10068E008CE599B4F906754E04123D8CE599D39418
:10069E00E54007E599C394F04002801685994F75A1
:1006AE004E027E017F00E54FC394E612687F8E32C4
:1006BE008F339007D0E4F0A3F0E599D394C44007AC
:1006CE00E599C394E64002802885994F754E0374D0
:1006DE00E5C3954FF533753200AE32AF3390627588
:1006EE0012684EE493F87401939007D0C8F0A3C833
:1006FE00F0D299020AB390006EE070429007D0E0FB
:10070E00FEA3E0FF74FFBE00039F5009EFC39446A3
:10071E00EE940640119007D0E0FEA3E0FFEFD394D5
:10072E006DEE940640139007D0E0FEA3E0FF90001C
:10073E008C1268A6E599F080038599738011900755
:10074E00D0E0FEA3E0FF90008C1268A6E599F09031
:10075E0007D012688D9007D0E0FEA3E0FFEFB40142
:10076E0006EEB40702800302089B90078CE0B43CAF
:10077E00028003020885C29C90006EE090012AF070
:10078E0090006FE0900099F0900070E09000B9F04A
:10079E00900071E09000E2F0900072E090008EF018
:1007AE00900073E09000D4F0900074E09000F2F0AE
:1007BE00900075E09000C6F0900076E09000E4F0B6
:1007CE00900077E0900114F0123769900080E0906D
:1007DE0000FBF0900081E09000B2F0900082E0907B
:1007EE0000B3F074639007CCF8E4F0E8A3F074ABB8
:1007FE00900057F0120448900057E4F075096475A4
:10080E0008001200E3A21F4038757201E572D394FE
:10081E0007502CE5729007CCF8E4F0E8A3F074AA28
:10082E00900057F012010FE572C394075009750935
:10083E00647508001200E37872740126F650CD80BC
:10084E0036757208E572D3940E502CE5729007CC73
:10085E00F8E4F0E8A3F074AA900057F012010FE547
:10086E0072C3940E50097509647508001200E3787E
:10087E0072740126F650CD74C89007CCF8E4F0E8F7
:10088E00A3F0D29C754E00754D007599FB020AB30C
:10089E009007D0E0FEA3E0FFEF4E7006859931750C
:1008AE0030009007D0E0FEA3E0FF74016F4E701B86
:1008BE00AC30AD31AA32AB33ED2BFBEC3AFA8A06F3
:1008CE008B0790008C1268A6E599F09007D01268FD
:1008DE008D9007D0E0FEA3E0FF74026F4E7021AC46
:1008EE0030AD3174566D4C7006E54F64E660028093
:1008FE0003123D8C123769854F99754E00754D0068
:10090E00020AB39007D0E0FEA3E0FF90008C1268BD
:10091E00A6E599F09007D012688D9007D0E0FEA35F
:10092E00E0FFAC32AD338F028E038C068D079062E2
:10093E00B712684EE493F9740193FEEAD39EEB99D5
:10094E004009854F99754E00754D00020AB3900708
:10095E00D0E0FEA3E0FF90008C1268A6E599F0901F
:10096E0007D012688D9007D0E0FEA3E0FFEFB40031
:10097E0006EEB401028003020AB3900067E075F040
:10098E0002A4FDACF08D72ED90008C1268B1EDFA00
:10099E00E0FBEA90008F1268B1EBFAE0FBEA2BFA6B
:1009AE00900067E0B502028003020AA50DED9000EB
:1009BE008C1268B1E572FDE0FAED9000901268B10C
:1009CE00EAFDE0FAEDC39AFD900067E0B5050280FE
:1009DE0003020AA5E57290008E1268B1E572FDE081
:1009EE00FAED9000911268B1EAFDE0FAED2AFD9061
:1009FE000067E0B505028003020AA5E57290009239
:100A0E001268B1FDE0FAED900067E0F4042A900060
:100A1E006EF0E5729000931268B1FDE0FAED900071
:100A2E0067E0F4042A90006FF0E57290009412686B
:100A3E00B1FDE0FAED900067E0F4042A900070F04A
:100A4E00E5729000951268B1FDE0FAED900067E056
:100A5E00F4042A9007CCF8E4F0E8A3F074AB90000D
:100A6E0057F01204487509647508001200E39007E8
:100A7E00CC12688D1204487509647508001200E3E3
:100A8E009007CC12688D1204487599F97509647532
:100A9E0008001200E380FE7599FF75096475080061
:050AAE001200E380FED0
:0F33F80002065902070402089E02091102095C2D
:100AB30022E54D903407F8282873020B989007D04D
:100AC300E0FEA3E0FF90005D1268A6E0F5999007B1
:100AD300D012688D9007D0E0FEA3E0FF74116F4E33
:100AE3007003754D00020B98856D99020B98900762
:100AF300D0E0FEA3E0FF90008C1268A6E0F599EF2A
:100B0300B40107EEB40703754D009007D012688D4A
:070B1300020B989007D1E0EE
:0F340700020ABD020AC0020AEB020AF1020B160A
:100B1A009035BAF82828738552998067855E99803E
:100B2A0062856099805D856499805885669980534D
:100B3A00856799804E85689980498569998044902E
:100B4A00001EE0F599803CA237B340077599FAC2B6
:100B5A00378017A228B3400575990F800B90005B68
:100B6A00E0F59990005BE4F0C2288017856A9980C5
:100B7A0012856599800D856B9980087599FC8003AB
:030B8A00754D00A6
:1035BA00020B21020B26020B2B020B30020B3502E7
:1035CA000B3A020B3F020B44020B49020B51020B4E
:0D35DA0076020B7B020B80020B85020B8A30
:0B0B8D009007D012688D80031235E73E
:03341600020B9511
:100B980022E537255AFFAE5950010E90008C126895
:100BA800A6E0F538E537255AFFAE5950010E0FBFBC
:100BB80000010E90008C1268A6E0F539853F3BE5F0
:100BC80038B539058538378041E539D39538401D22
:100BD800E539C39538853AF0A4FFAEF0E53B8E04BD
:100BE8008F05FF12686FED2538F537801DE538C38E
:100BF8009539853AF0A4FFAEF0E53B8E048F05FFEA
:100C080012686FEDF4042538F53722E539D39538A5
:100C1800401DE539C39538853AF0A4FFAEF0E53BB1
:100C28008E048F05FF12686FED2538F537801DE5B6
:100C380038C39539853AF0A4FFAEF0E53B8E048FB2
:100C480005FF12686FEDF4042538F53722900092FD
:100C5800E0B40170E56675F00A84FF7E008F37E521
:100C68006675F00A84ADF07C008D3A753F0A7559B7
:100C780005755A24E537C394115005120B9980065F
:100C88009005C1E0F537E537900085F0E56675F029
:100C98000A84FF7E008F37E56675F00A84ADF07C24
:100CA800008D3A753F0A755905755A5AE537C39448
:100CB800115005120B9980069005F7E0F537E537D6
:100CC800900016F022900092E0B4016AE56675F093
:100CD8000A84FF7E008F37E56675F00A84ADF07CE4
:100CE800008D3A753F0A755905755A36E537C3942C
:100CF800115005120B9980069005D3E0F53785371A
:100D08004BE56675F00A84FF7E008F37E56675F05F
:100D18000A84ADF07C008D3A753F0A755905755AFD
:100D280048E537C394115005120B9980069005E5E4
:100D3800E0F53785374C22E55E75F00484FF7E00C8
:100D48008F37E55E75F00484ADF07C008D3A753F11
:100D580004755901755A00E537C3943F5005120BC5
:100D68009980069001CBE0F53785372975280090E2
:100D7800005AE075F020A4FFAEF09000DDE08E048C
:100D88008F05FF12686F8D379000C5E0D3955E50D0
:100D980003020E459000E9E0D3955E4010ED900106
:100DA800CC1268B1E0F52B752A00020E429000B40F
:100DB800E0D3955E4043E5379001CC1268B1E0F589
:100DC80038E5379001EC1268B1E0F5399000E9E0B8
:100DD800F404255EF53A9000B4E0FE9000E9E0F4F2
:100DE800042EF53BE538B539058538378003120CF4
:100DF8001385372B752A008041E5379001EC12687E
:100E0800B1E0F538E53790020C1268B1E0F5399099
:100E180000B4E0F404255EF53A9000C5E0FE9000C9
:100E2800B4E0F4042EF53BE538B53905853837804C
:100E380003120C1385372B752A00020EEC9000EC78
:100E4800E0D3955E5011E53790024C1268B1E0F599
:100E58002B752A00020EEC9000B5E0D3955E504346
:100E6800E53790022C1268B1E0F538E53790024C6E
:100E78001268B1E0F5399000B5E0F404255EF53A62
:100E88009000ECE0FE9000B5E0F4042EF53BE53868
:100E9800B539058538378003120C1385372B752A29
:100EA800008041E53790020C1268B1E0F538E5376B
:100EB80090022C1268B1E0F5399000C5E0F40425E1
:100EC8005EF53A9000B5E0FE9000C5E0F4042EF51A
:100ED8003BE538B539058538378003120C1385375B
:100EE8002B752A00229000FDE0F53C753F117559DD
:100EF80002755A00AE51AF52E53C75F00FA4FDAC37
:100F0800F0EDD39FEC9E4021E53C8E048F05FF1247
:100F1800686FED75F010A4FFAEF0E55E75F0118412
:100F2800FD7C00ED2FF53D800EE55E75F01184FF28
:100F38007E00EF24F0F53D853D37E55E75F01184C0
:100F4800AFF07E008F3A120B9985373EAE51AF5203
:100F58009000FDE075F00FA4FDACF0EDD39FEC9E82
:100F68004028755902755A10853D37120B99853EF0
:100F780038853739AE51AF52E53C8E048F05FF12E4
:100F8800689A8D3A853C3B120C13853729752800E1
:100F9800752B64752A00229000FDE0F53C753F1121
:100FA800755902755A00AE51AF52E53C75F00FA461
:100FB800FDACF0EDD39FEC9E4021E53C8E048F05FF
:100FC800FF12686FED75F010A4FFAEF0E56075F0E4
:100FD8001184FD7C00ED2FF53D800EE56075F01164
:100FE80084FF7E00EF24F0F53D853D37E56075F020
:100FF8001184AFF07E008F3A120B9985373EAE51BF
:10100800AF529000FDE075F00FA4FDACF0EDD39F5A
:10101800EC9E4028755902755A10853D37120B9978
:10102800853E38853739AE51AF52E53C8E048F0581
:10103800FF12689A8D3A853C3B120C138537297547
:1010480028009000C7E0B40453E55E75F00484FFFF
:101058007E008F37E55E75F00484ADF07C008D3A34
:10106800753F04755901755A00E537C3943F50051B
:10107800120B9980069001CBE0F537AE28AF29E531
:101088003712687F74648E048F05FF12686FAE286C
:10109800AF29EF2DFDEE3CFC8C288D29752B64754E
:1010A8002A0022900092E0B40146E56675F00A84B1
:1010B800FF7E008F37E56675F00A84ADF07C008D01
:1010C8003A753F0A755905755A00E537C3941150AA
:1010D80005120B99800690059DE0F537AE2AAF2BD7
:1010E800E5372FFF50010E74641268C38E2A8F2BC8
:1010F800900093E0B40146E56775F00A84FF7E002E
:101108008F37E56775F00A84ADF07C008D3A753F3E
:101118000A755905755A6CE537C394115005120BB9
:10112800998006900609E0F537AE2AAF2BE5372FF0
:10113800FF50010E74641268C38E2A8F2B9000A290
:10114800E0B40249E569C3944175F00584FF7E0067
:101158008F37E56975F00584ADF07C008D3A753FF1
:1011680005755906755A00E537C394135005120BD7
:1011780099800690069FE0F537AE2AAF2BE5372F0A
:10118800FF50010E74641268C38E2A8F2B9000E4FE
:10119800E0B40202800302124AE55E75F01584FF8E
:1011A8007E008F37E55E75F01584ADF07C008D3AD2
:1011B800753F15755903755AF4E537C3940B5005F7
:1011C800120B99800690048BE0F537E53775F0FF30
:1011D800A4FFAEF09000E5E08E048F05FF12686F63
:1011E800ED90007EF0E56575F078A4FFAEF074FF31
:1011F8008E048F05FF12686F8C598D5A74028C0605
:101208008D071200398F37AC59AD5A7404FF126834
:101218009A8D3A753F04755906755A28E537C3946F
:101228001D5005120B9980069006D1E0F537AE2ABD
:10123800AF2BE5372FFF50010E74641268C38E2A56
:101248008F2B900091E0B4025DE56075F064A4FF17
:10125800AEF074081200398E5B8F5C74058E048FB3
:1012680005FF12686F8D37AE5BAF5C74058E048F17
:1012780005FF12689A8D3A753F05755905755ADE4E
:10128800E537C394135005120B99800690067DE04C
:10129800F537AE2AAF2BE5372FFF50010E746412D5
:1012A80068C38E2A8F2B9000D3E0703C90005AE0E0
:1012B80075F00584FF7E008F3790005AE075F005C1
:1012C80084ADF07C008D3A753F05755905755AC097
:1012D800E537C3941D5005120B998006900669E006
:1012E800F537E537900086F02290009AE0B40117B0
:1012F8009007D3E0252BFFAE2A50010E9000EEE0B8
:101308001268C38E2A8F2B900112E0B40114900149
:1013180013E0A851B8000495525007E55EC3955FE5
:10132800400280129000BCE0252BFFAE2A50010E2F
:101338008E2A8F2B802F90009AE0B40316A22AB32E
:10134800B350109007D6E0C39405A851B80006958D
:1013580052400280109000BCE0252BFFAE2A5001BD
:101368000E8E2A8F2B900094E0B40202800302159F
:101378004D900097E0602FE566D394464028900092
:1013880017E0FEA3E0FF9000D2E075F003A4FDACE7
:10139800F0EFD39DEE9C400E9000F6E0A851B80007
:1013A80005D39552500302154D9000DFE0855EF09D
:1013B800A4FFAEF0740512687F74071200398E59C5
:1013C8008F5A90009EE0A851B80004955250129090
:1013D800009FE075F002A4FDACF0EFC39DEE9C40C9
:1013E8000302154DE55E75F00B84FF7E0090061C28
:1013F8001268A6FEE0FFEE900096E0FEEF8E0088F1
:10140800F0A4FFAEF074648E048F05FF12686F8C31
:10141800598D5A90005AE075F018A4FFAEF090006C
:10142800DDE08E048F05FF12686F8C068D0790062D
:10143800341268A6AE59AF5AE012687F74648E04FD
:101448008F05FF12686F8C598D5AE564A859B8004A
:1014580077D3955A4072E564C3955AFFE49559FECF
:101468008E598F5A7428BE00039F500C755A2875E0
:101478005900740D90005BF0AE59AF5A900097E098
:1014880012687F74288E048F05FF12686F8C598D3F
:101498005AAE28AF29740A8E048F05FF12686F8D23
:1014A800068C07AC59AD5ACFCECF120003740A8E02
:1014B800048F05FF12686F8C598D5AAE28AF291218
:1014C80068CB8E288F29807DE564A859B8000495DB
:1014D8005A5072AE59AF5AE5641268C38E598F5A82
:1014E8007428BE00039F500C755A28755900740D56
:1014F80090005BF0AE59AF5A900097E012687F7485
:10150800288E048F05FF12686F8C598D5AAE28AF4C
:1015180029740A8E048F05FF12686F8D068C07AC3C
:1015280059AD5ACFCECF120003740A8E048F05FF2F
:1015380012686F8C598D5AAE28AF29EF2DFDEE3CFD
:10154800FC8C288D29229000F2E0B4026AE55E75D1
:10155800F00884FF7E008F37E55E75F00884ADF0F3
:101568007C008D3A753F08755901755AE0E537C317
:10157800943F5005120B99800690028BE0F5378551
:10158800372D752C00AE2CAF2DAC2AAD2B120003D5
:1015980074648E048F05FF12686F8C2C8D2D90005B
:1015A8008FE08C068D0712687F74648E048F05FFA8
:1015B80012686F8C2C8D2DAE28AF29AC2AAD2B125A
:1015C800000374648E048F05FF12686F8C288D29C0
:1015D80090008FE08C068D0712687F74648E048FEC
:1015E80005FF12686F8C288D29A20A401DAE51AFE5
:1015F800527405BE00039F5002D20AE560D394CC12
:101608004008D201741190005BF09000F1E0B40240
:10161800089000F3E0640160028035AE28AF29E548
:101628006A12687F74E78E048F05FF12686F8C2832
:101638008D299000F2E0B40217AE2CAF2DE56A12A6
:10164800687F74E78E048F05FF12686F8C2C8D2DD0
:101658009000B1E05402601B9000A8E0A851B800C7
:1016680012D39552400DA20AB3B35007E560C39454
:101678009A40028028AE35AF369000A6E075F00299
:10168800A4FDACF0EF2DFDEE3CFC74022DFD5001E5
:101698000CE560BC0007D39D4003754301856036A7
:1016A800753500E5437003021791900104E0C39576
:1016B800435003021783900114E0C394025076E567
:1016C8006675F00A84FF7E0090058C1268A6E0F526
:1016D8005A755900AE59AF5A9000A7E012687F7446
:1016E800648E048F05FF12686F8C5B8D5C9001041B
:1016F800E004C395438C068D0712687F900104E0CF
:101708008E048F05FF12686F8C5B8D5CAE28AF2945
:10171800EF2DFDEE3CFC8C288D299000F2E0B40200
:1017280012AE2CAF2DAA5BAB5CEF2BFBEE3AFA8A1C
:101738002C8B2D8046900104E004C39543854BF023
:10174800A4FFAEF0900104E08E048F05FF12686FCD
:101758008C5B8D5CAE28AF29EF2DFDEE3CFC8C2810
:101768008D299000F2E0B40212AE2CAF2DAA5BAB2B
:101778005CEF2BFBEE3AFA8A2C8B2D054390010483
:10178800E0C3954350037543009000B1E0540160F5
:101798001B9000A5E0A851B80012D39552400DA2A5
:1017A8000AB3B35007E55EC394CC4002802590008D
:1017B800A3E075F003A4FFAEF0E5402FFF50010E43
:1017C80074032FFF50010EE55EBE0007D39F400350
:1017D800754401855E40E54470030218C490010514
:1017E800E0C3954450030218B6900114E0C3940274
:1017F8005076E56675F00A84FF7E0090058C1268C5
:10180800A6E0F55A755900AE59AF5A9000A4E012F7
:10181800687F74648E048F05FF12686F8C5B8D5C23
:10182800900105E004C395448C068D0712687F90EB
:101838000105E08E048F05FF12686F8C5B8D5CAE2E
:1018480028AF29EF2DFDEE3CFC8C288D299000F265
:10185800E0B40212AE2CAF2DAA5BAB5CEF2BFBEE13
:101868003AFA8A2C8B2D8046900105E004C39544F2
:10187800854CF0A4FFAEF0900105E08E048F05FFC3
:1018880012686F8C5B8D5CAE28AF29EF2DFDEE3CA6
:10189800FC8C288D299000F2E0B40212AE2CAF2DFA
:1018A800AA5BAB5CEF2BFBEE3AFA8A2C8B2D054436
:1018B800900105E0C395445003754400900107E08A
:1018C8002529FFAE2850010E8E288F299000B6E0FA
:1018D800A828B80004952950099000B6E0F52975A4
:1018E80028009000F2E0B4020D9000B6E0A82CB8F1
:1018F8000006952D400280099000B6E0F52D752C64
:1019080000229000F2E0B401028003021A15A20A34
:10191800B35003021A139000BDE0B40168AE28AFBB
:1019280029AC51AD52120003743C8E048F05FF128E
:10193800686F9000CDE0BC00109D400D9000CFE096
:10194800A828B8000495295002D202AE28AF29ACC5
:1019580051AD52120003743C8E048F05FF12686F5C
:101968009000CDE0C3940ABC0015D39D40119000AF
:10197800CFE0C39405A828B80005D3952950028064
:1019880002C2028068AE28AF29AC51AD52120003E2
:1019980074788E048F05FF12686F9000CDE0BC004C
:1019A800109D400D9000CFE0A828B800049529505C
:1019B80004D2028038AE28AF29AC51AD52120003D0
:1019C80074788E048F05FF12686F9000CDE0C39481
:1019D8000ABC0015D39D40119000CFE0C39405A820
:1019E80028B80005D3952950028002C202A202B38A
:1019F8004019AE28AF299000CEE012687F74648E3B
:101A0800048F05FF12686F8C288D298002C202A2FC
:101A180000B34006A201B3B3500990001DE4F0A33F
:101A2800F08024AE28AF297400D39F74019E400C27
:101A380090001DE528F0A3E529F0800B74FF9000C5
:101A48001DF8E4F0E8A3F09000D4E0D39402400C31
:101A58009000BFE07006A20AB3B34002801AAE2815
:101A6800AF29740212687F8E288F29AE2CAF2D748F
:101A78000212687F8E2C8F2D9000BDE0B4011AAE43
:101A880028AF29740212687F8E288F29AE2CAF2DBB
:101A9800740212687F8E2C8F2DAE28AF29745E12C7
:101AA800687F740A8E048F05FF12686F8C288D2951
:101AB8009000F2E0B40217AE2CAF2D745E12687F6E
:101AC800740A8E048F05FF12686F8C2C8D2DAE283A
:101AD800AF297402BE000AD39F40067529027528F3
:101AE80000AE2CAF2D7402BE000AD39F4006752DA0
:101AF80002752C0090001BE528F0A3E529F0229040
:101B0800005AE090038C1268B1E0F5417542649088
:101B1800005AE0FE9000C8E0D39E4037E55E75F0BD
:101B28000884FF7E008F37E55E75F00884ADF07C91
:101B3800008D3A753F08755903755A96E537C39471
:101B48001F5005120B998006900441E0F537853740
:101B5800428035E55E75F00884FF7E008F37E55ECC
:101B680075F00884ADF07C008D3A753F087559030F
:101B7800755AB6E537C3941F5005120B9980069025
:101B88000461E0F537853742229000FEE0F53C75A8
:101B98003F11755904755A00AE51AF52E53C75F0C6
:101BA8000FA4FDACF0EDD39FEC9E4021E53C8E04E4
:101BB8008F05FF12686FED75F010A4FFAEF0E55EBB
:101BC80075F01184FD7C00ED2FF53D800EE55E7506
:101BD800F01184FF7E00EF24F0F53D853D37E55E8A
:101BE80075F01184AFF07E008F3A120B9985373E5D
:101BF800AE51AF529000FEE075F00FA4FDACF0EDD1
:101C0800D39FEC9E4028755904755A10853D3712AC
:101C18000B99853E38853739AE51AF52E53C8E0475
:101C28008F05FF12689A8D3A853C3B120C13853755
:101C380041754264229000FEE0F53C753F117559EC
:101C480004755A00AE51AF52E53C75F00FA4FDACD7
:101C5800F0EDD39FEC9E4021E53C8E048F05FF12EA
:101C6800686FED75F010A4FFAEF0E56075F01184B3
:101C7800FD7C00ED2FF53D800EE56075F01184FFC9
:101C88007E00EF24F0F53D853D37E56075F0118461
:101C9800AFF07E008F3A120B9985373EAE51AF52A6
:101CA8009000FEE075F00FA4FDACF0EDD39FEC9E24
:101CB8004028755904755A10853D37120B99853E91
:101CC80038853739AE51AF52E53C8E048F05FF1287
:101CD800689A8D3A853C3B120C13853741754264EE
:101CE8009000F9E0B4047990005AE0FE9000C8E052
:101CF800D39E4037E55E75F00884FF7E008F37E598
:101D08005E75F00884ADF07C008D3A753F08755912
:101D180003755A96E537C3941F5005120B99800630
:101D2800900441E0F5378537428035E55E75F00867
:101D380084FF7E008F37E55E75F00884ADF07C0087
:101D48008D3A753F08755903755AB6E537C3941F20
:101D58005005120B998006900461E0F537853742EB
:101D680022900092E0B4013BE56675F00A84FF7E9C
:101D7800008F37E56675F00A84ADF07C008D3A7502
:101D88003F0A755905755A12E537C3941150051263
:101D98000B9980069005AFE0F537E5422537C394E7
:101DA80064F542900093E0B4013BE56775F00A845E
:101DB800FF7E008F37E56775F00A84ADF07C008DF3
:101DC8003A753F0A755905755A7EE537C39411501F
:101DD80005120B99800690061BE0F537E54225377A
:101DE800C39464F542E5412542F53490009AE0B485
:101DF80002109007D2E02534FE9000EEE0F4042EA5
:101E0800F5349000F1E0D394014040E56AC394E7CB
:101E1800501D74E7C3956AFE9007D4E08E00F5F074
:101E2800E884FF7E008F37E5342537F534801CE5DC
:101E38006AC394E7FE9007D4E08E00F5F0E884FFCB
:101E48007E008F37E534C39537F534A20A4006E59E
:101E5800412464F534E534D394644009E534C394EB
:101E680064F53480037534009000CAE0C39534509B
:101E7800069000CAE0F53422D200900084E0A85110
:101E8800B8000495525041900084E0A851B800046D
:101E98009552500375340F900084E004A851B8009F
:101EA800049552500375340A900084E02402A85126
:101EB800B8000495525005753405C200900084E0BE
:101EC8006006740990005BF0C23A7E017F009000C2
:101ED800D0E012687F9000DFE08E048F05FF126863
:101EE8006FE55EBC0017D39D40139000D9E0B402A3
:101EF80004D23A8002C200740A90005BF09000D1CC
:101F0800E0C3956650159000E3E0A851B800049529
:101F1800525002C200740B90005BF0E566C39464F3
:101F2800501D900129E0600D900129E0A851B800EA
:101F380006955240028008C200740B90005BF0A224
:101F4800004003753405900112E0B40114900113A8
:101F5800E0A851B8000495525007E55EC3955F406C
:101F68000280089000BBE0F534803A90009AE0B413
:101F78000306A22AB3B34002802B9007D6E0C3948D
:101F880005A851B800049552500C9000BBE0F534F8
:101F9800740C90005BF09007D6E0A851B800049547
:101FA800525002C20085346B90008CE02534FE90BC
:101FB800005AE075F01E84FC7F00EE2CF534229068
:101FC800005AE075F00584FF7E008F3790005AE0D4
:101FD80075F00584ADF07C008D3A753F05755903A1
:101FE800755AD69000DDE01475F00584FF7E00E593
:101FF80037BE00039F5005120B99800BE5379004FC
:10200800621268B1E0F537E5379007D5F09007D54B
:10201800E0FE9000CCE0C39E50089000CCE0900712
:10202800D5F022E56675F00A84FF7E0090058C12D3
:1020380068A6E0F546E546D394644010E546C394A7
:102048006475F00F84FF7E008F468003754600900C
:1020580000AFE02546F546229007C6E0FEA3E0FF64
:102068007404120039E55E12687F740F8E048F05C0
:10207800FF12686F9007C4ECF0A3EDF09000A2E0A7
:10208800B40262E569C3944175F00584FF7E008F50
:1020980037E56975F00584ADF07C008D3A753F052C
:1020A800755906755A14E537C394175005120B99DC
:1020B80080069006B3E0F5379007C4E0FEA3E0FF82
:1020C800740A8E048F05FF12686FE5378C068D073A
:1020D80012687F740A8E048F05FF12686F9007C418
:1020E800ECF0A3EDF09007C4E0FEA3E0FF9007CA70
:1020F800E0FCA3E0FDEDD39FEC9E400F9007CAE003
:10210800F8A3E09007C4C8F0A3C8F0229006D3E073
:10211800903419F8282873804C85527280479000B3
:10212800DFE0855EF0A4FFAEF074081200398F720C
:102138008033856072802E856672802985677280FB
:1021480024856872801F856972801A856A72801575
:102158008565728010856472800B856B728006902D
:05216800001EE0F5720D
:1034190002211F02212102212602213A02213F0213
:10342900214402214902214E02215302215802213D
:073439005D02216202216720
:10216D009006D4E0FE9006D5E0D39E404B9006D36A
:10217D00E0B404189006D5E0C395725002D22B90AE
:10218D0006D4E0D395724002C22B802A9006D4E08B
:10219D00C3957250099006D5E0D395725002800216
:1021AD00D22B9006D4E0D3957250099006D5E0C39A
:1021BD0095725002C22B802A9006D4E0D3957240BE
:1021CD00099006D5E0C3957240028002C22B90069D
:1021DD00D4E0C3957240099006D5E0D395724002C4
:1021ED00D22B229006D7E0903440F8282873804CEB
:1021FD0085527280479000DFE0855EF0A4FFAEF05F
:10220D0074081200398F728033856072802E856656
:10221D007280298567728024856872801F85697236
:10222D00801A856A7280158565728010856472804A
:0C223D000B856B72800690001EE0F572AD
:103440000221FB0221FD02220202221602221B029D
:10345000222002222502222A02222F0222340222C4
:073460003902223E02224363
:102249009006D8E0FE9006D9E0D39E405F9006D76D
:10225900E0B404189006D9E0C395725002D22C90CC
:1022690006D8E0D395724002C22C803E9006D8E091
:10227900C3957250099006D9E0D395725002800235
:10228900D22C9006D8E0D3957250099006D9E0C3B4
:1022990095725002C22C9006D7E0B401099000EB68
:1022A900E0D3956050028002C22C802A9006D8E0C3
:1022B900D3957240099006D9E0C395724002800215
:1022C900C22C9006D8E0C3957240099006D9E0D394
:1022D90095724002D22C229006DBE0903467F828F0
:1022E9002873804C85527280479000DFE0855EF04C
:1022F900A4FFAEF074081200398F728033856072C2
:10230900802E85667280298567728024856872802F
:102319001F856972801A856A7280158565728010B9
:10232900856472800B856B72800690001EE0F572E1
:103467000222EB0222ED0222F202230602230B02C2
:10347700231002231502231A02231F0223240223E7
:073487002902232E0223336A
:102339009006DCE0FE9006DDE0D39E404B9006DB84
:10234900E0B404189006DDE0C395725002D22D90D6
:1023590006DCE0D395724002C22D802A9006DCE0AB
:10236900C3957250099006DDE0D395725002800240
:10237900D22D9006DCE0D3957250099006DDE0C3BA
:1023890095725002C22D802A9006DCE0D3957240E6
:10239900099006DDE0C3957240028002C22D9006C5
:1023A900DCE0C3957240099006DDE0D395724002E6
:1023B900D22D229006DFE090348EF8282873804CC5
:1023C90085527280479000DFE0855EF0A4FFAEF091
:1023D90074081200398F728033856072802E856689
:1023E9007280298567728024856872801F85697269
:1023F900801A856A7280158565728010856472807D
:0C2409000B856B72800690001EE0F572DF
:10348E000223C70223C90223CE0223E20223E7024C
:10349E0023EC0223F10223F60223FB022400022472
:0734AE000502240A02240FAD
:102415009006E0E0FE9006E1E0D39E404B9006DF9B
:10242500E0B404189006E1E0C395725002D22E90F4
:1024350006E0E0D395724002C22E802A9006E0E0C5
:10244500C3957250099006E1E0D39572500280025F
:10245500D22E9006E0E0D3957250099006E1E0C3D4
:1024650095725002C22E802A9006E0E0D395724004
:10247500099006E1E0C3957240028002C22E9006E3
:10248500E0E0C3957240099006E1E0D39572400201
:10249500D22E229006E3E09034B5F8282873804CBC
:1024A50085527280479000DFE0855EF0A4FFAEF0B4
:1024B50074081200398F728033856072802E8566AC
:1024C5007280298567728024856872801F8569728C
:1024D500801A856A728015856572801085647280A0
:0C24E5000B856B72800690001EE0F57203
:1034B5000224A30224A50224AA0224BE0224C302D4
:1034C50024C80224CD0224D20224D70224DC0224FB
:0734D500E10224E60224EBF2
:1024F1009006E4E0FE9006E5E0D39E404B9006E3B3
:10250100E0B404189006E5E0C395725002D22F9012
:1025110006E4E0D395724002C22F802A9006E4E0DF
:10252100C3957250099006E5E0D39572500280027E
:10253100D22F9006E4E0D3957250099006E5E0C3EE
:1025410095725002C22F802A9006E4E0D395724022
:10255100099006E5E0C3957240028002C22F900601
:10256100E4E0C3957240099006E5E0D3957240021C
:10257100D22F229006E7E09034DCF8282873804CB3
:1025810085527280479000DFE0855EF0A4FFAEF0D7
:1025910074081200398F728033856072802E8566CF
:1025A1007280298567728024856872801F856972AF
:1025B100801A856A728015856572801085647280C3
:0C25C1000B856B72800690001EE0F57226
:1034DC0002257F02258102258602259A02259F025C
:1034EC0025A40225A90225AE0225B30225B8022582
:0734FC00BD0225C20225C735
:1025CD009006E8E0FE9006E9E0D39E404B9006E7CA
:1025DD00E0B404189006E9E0C395725002D2309031
:1025ED0006E8E0D395724002C230802A9006E8E0FA
:1025FD00C3957250099006E9E0D39572500280029E
:10260D00D2309006E8E0D3957250099006E9E0C308
:10261D0095725002C230802A9006E8E0D395724040
:10262D00099006E9E0C3957240028002C23090061F
:10263D00E8E0C3957240099006E9E0D39572400237
:10264D00D230229006EBE0903503F8282873804CA9
:10265D0085527280479000DFE0855EF0A4FFAEF0FA
:10266D0074081200398F728033856072802E8566F2
:10267D007280298567728024856872801F856972D2
:10268D00801A856A728015856572801085647280E6
:0C269D000B856B72800690001EE0F57249
:1035030002265B02265D02266202267602267B02E3
:10351300268002268502268A02268F022694022608
:073523009902269E0226A377
:1026A9009006ECE0FE9006EDE0D39E404B9006EBE1
:1026B900E0B404189006EDE0C395725002D231904F
:1026C90006ECE0D395724002C231802A9006ECE014
:1026D900C3957250099006EDE0D3957250028002BD
:1026E900D2319006ECE0D3957250099006EDE0C323
:1026F90095725002C231802A9006ECE0D39572405F
:10270900099006EDE0C3957240028002C23190063D
:10271900ECE0C3957240099006EDE0D39572400252
:10272900D231229006EFE090352AF8282873804CA0
:1027390085527280479000DFE0855EF0A4FFAEF01D
:1027490074081200398F728033856072802E856615
:102759007280298567728024856872801F856972F5
:10276900801A856A72801585657280108564728009
:0C2779000B856B72800690001EE0F5726C
:10352A0002273702273902273E022752022757026B
:10353A00275C02276102276602276B02277002278F
:07354A007502277A02277FBA
:102785009006F0E0FE9006F1E0D39E404B9006EFF8
:10279500E0B404189006F1E0C395725002D232906D
:1027A50006F0E0D395724002C232802A9006F0E02E
:1027B500C3957250099006F1E0D3957250028002DC
:1027C500D2329006F0E0D3957250099006F1E0C33D
:1027D50095725002C232802A9006F0E0D39572407D
:1027E500099006F1E0C3957240028002C23290065C
:1027F500F0E0C3957240099006F1E0D3957240026E
:10280500D232229006F3E0903551F8282873804C97
:1028150085527280479000DFE0855EF0A4FFAEF040
:1028250074081200398F728033856072802E856638
:102835007280298567728024856872801F85697218
:10284500801A856A7280158565728010856472802C
:0C2855000B856B72800690001EE0F5728F
:1035510002281302281502281A02282E02283302F3
:10356100283802283D02284202284702284C022816
:073571005102285602285BFD
:102861009006F4E0FE9006F5E0D39E404B9006F30F
:10287100E0B404189006F5E0C395725002D233908B
:1028810006F4E0D395724002C233802A9006F4E048
:10289100C3957250099006F5E0D3957250028002FB
:1028A100D2339006F4E0D3957250099006F5E0C357
:1028B10095725002C233802A9006F4E0D39572409B
:1028C100099006F5E0C3957240028002C23390067A
:1028D100F4E0C3957240099006F5E0D39572400289
:1028E100D233229006F7E0903578F8282873804C8F
:1028F10085527280479000DFE0855EF0A4FFAEF064
:1029010074081200398F728033856072802E85665B
:102911007280298567728024856872801F8569723B
:10292100801A856A7280158565728010856472804F
:0C2931000B856B72800690001EE0F572B2
:103578000228EF0228F10228F602290A02290F027E
:10358800291402291902291E02292302292802299D
:073598002D02293202293740
:10293D009006F8E0FE9006F9E0D39E404B9006F726
:10294D00E0B404189006F9E0C395725002D23490A9
:10295D0006F8E0D395724002C234802A9006F8E062
:10296D00C3957250099006F9E0D39572500280021A
:10297D00D2349006F8E0D3957250099006F9E0C371
:10298D0095725002C234802A9006F8E0D3957240B9
:10299D00099006F9E0C3957240028002C234900698
:1029AD00F8E0C3957240099006F9E0D395724002A4
:1029BD00D23422AE2EAF2F74F5D39F74019E4008F2
:1029CD00782E1268D3022ADA752F01752E00AE51BA
:1029DD00AF52E546BE000DD39F40099000C1E0D334
:1029ED00954740028023754700E546C39552F57221
:1029FD009000C4E0D395454008E5452572F5458026
:102A0D00069000C4E0F5458002054790009DE0D397
:102A1D009560401CE55EC3955F4015AE51AF52E524
:102A2D0046BE00039F50099000C2E0D39548400276
:102A3D00806E9007D9E0A851B800049552500375E7
:102A4D004A009007D9E0A851B8000BD39552400623
:102A5D00E5529007D9F0E54A7041E552C39546F528
:102A6D0072E572D3940540037572059000C3E0C3FF
:102A7D0095455007E572C3954540028009E545C36C
:102A8D009572F54580069000C3E0F5459000C3E0D2
:102A9D00D3954540069000C3E0F54575480080028A
:102AAD000548E54A701690009DE0C39560500DE510
:102ABD00462405A851B8000695524002800F90009B
:102ACD00B0E0F545754A0174789007D9F022AE2E25
:102ADD00AF2F74E9D39F74039E4008782E1268D3EC
:102AED00022C79752F01752E00754532A235402ABD
:102AFD007545199000B0E075F002A4FFAEF0E54702
:102B0D00BE0006D39F4002D2350547754A0374783F
:102B1D009007D9F0754900022C68AE51AF52E546C9
:102B2D006F4E7003022C68E546BE000DD39F400921
:102B3D009000C1E0D395474002800F754700E54AEC
:102B4D00C394035003754519800DE546C39552F5A1
:102B5D0072E5472572F54790009DE0D39560400ED4
:102B6D009007D9E0A851B80007D395524002800CC8
:102B7D0005499000B0E0B54903754A00E54AB40334
:102B8D0006A20AB3B34002800A0549E549B43C03E5
:102B9D00754A02E54AB402299007D9E0A851B80058
:102BAD000ED395524009E5529007D9F07549009022
:102BBD00009DE0C39560500975490074789007D960
:102BCD00F0E54A705A90009DE0D39560401CE55E9B
:102BDD00C3955F4015AE51AF52E546BE00039F5001
:102BED00099000C2E0D395484002800875480075F1
:102BFD00454B8028E552C39546F572E572D3940591
:102C0D00400375720590009DE0D395604008E5483E
:102C1D002572F5488006E5482406F548754900E516
:102C2D004A701690009DE0C39560500DE546240551
:102C3D00A851B80006955240028003754A01E54A35
:102C4D00B4011875451905499000B0E0B5490675F0
:102C5D004A0275490074789007D9F0E54575F00A78
:102C6D00A4FFAEF09007CEEEF0A3EFF022E56E904C
:102C7D00359FF8282873900095E07003022E289058
:102C8D0000CBE0B401028003022D78900058E0B52E
:102C9D005D028003022D757E017F00E5BE12687F07
:102CAD00E5BD2FFF50010E8E598F5A741012687F9B
:102CBD00900083E08E048F05FF12686F9007DAECA9
:102CCD00F0A3EDF0E56A60089000F1E064026002A7
:102CDD0080269000F3E0B4011F9007DAE0FEA3E038
:102CED00FF74E712687FE56A8E048F05FF12686F27
:102CFD009007DAECF0A3EDF0900095E0B402279088
:102D0D0007DCE0FEA3E0FF9007DAE0FCA3E0FDEFB7
:102D1D002DFDEE3CFC74018C068D071200399007D9
:102D2D00DAEEF0A3EFF09007DAE0FEA3E0FF9007F4
:102D3D00DCE0FCA3E0FDEDD39FEC9E4004D2388097
:102D4D0002B2389007DAE0F8A3E09007DCC8F0A3F0
:102D5D00C8F09000C7E064016006A238B3B340022A
:102D6D0080069007DBE0F55E022E26D2387E017FCD
:102D7D0000E5BE12687FE5BD2FFF50010E8E598F05
:102D8D005A741012687F900083E08E048F05FF1235
:102D9D00686F9007DAECF0A3EDF0E56A600890003B
:102DAD00F1E06402600280269000F3E0B4011F9010
:102DBD0007DAE0FEA3E0FF74E712687FE56A8E0490
:102DCD008F05FF12686F9007DAECF0A3EDF090001D
:102DDD0095E0B402279007DCE0FEA3E0FF9007DA50
:102DED00E0FCA3E0FDEF2DFDEE3CFC74018C068DA7
:102DFD00071200399007DAEEF0A3EFF09007DAE052
:102E0D00F8A3E09007DCC8F0A3C8F09000C7E06419
:102E1D000160069007DBE0F55E8003755E009000B3
:102E2D0091E07006756E01022C7A75BB180233F3B2
:102E3D00900091E07003022FC97E017F00E5BE1264
:102E4D00687FE5BD2FFF50010E8E598F5A9000D728
:102E5D00E0B4010F7E0F7FFFAC59AD5A1268CB8ED7
:102E6D00598F5A9000FCE0B40245AE59AF5A90000C
:102E7D0027E0FCA3E0FDEDD39FEC9E400A900027D8
:102E8D00E559F0A3E55AF0AE59AF5A900029E0FC90
:102E9D00A3E0FDEFD39DEE9C400A900029E559F08B
:102EAD00A3E55AF0AE59AF5A74041200398F6090F1
:102EBD0000FCE0704CAE59AF5A900027E0FCA3E047
:102ECD00FDEFD39DEE9C40091268CB8E598F5A8031
:102EDD0006755A00755900AE59AF5A741012687FB5
:102EED00900080E08E048F05FF12686F8C598D5A0B
:102EFD0074FFBC0009D39D4005855A608003756041
:102F0D00FE9000C7E0B401028003022FC7A20AB3EE
:102F1D00B3500E90009BE0A851B80005D3955250C8
:102F2D0003022FBC90009CE075F019A4FFAEF09049
:102F3D0000DFE08E048F05FF12686F9000D8E085EA
:102F4D0060F0A4FFAEF074648D028C038E048F05C7
:102F5D00FF12686FEA2DFDEB3CFC8C598D5AE56A2A
:102F6D00600F9000F1E0B402089000F3E06401609E
:102F7D00028017AE59AF5A74E712687FE56A8E0466
:102F8D008F05FF12686F8C598D5AAE59AF5A900745
:102F9D00DAE0FCA3E0FDEDD39FEC9E4005855A5E83
:102FAD00800BA238B340069007DBE0F55E800BA2E4
:102FBD0038B340069007DBE0F55E80037560009046
:102FCD000094E07006756E02022C7A75BB190233FF
:102FDD00F3900094E0700302307EE55DD395504090
:102FED000302307C900025E0FEA3E0FFE56412684B
:102FFD00C3900025EEF0A3EFF07E017F00E5BE1239
:10300D00687FE5BD2FFF50010E8E598F5A9001013B
:10301D00E07013740A12687F74518E048F05FF12CD
:10302D00686F8D648019AE59AF5A740A12687F8F1C
:10303D00048E057E017F95CDCCCD12676D8F64E535
:10304D0064D394644003756464900025E0FEA3E0AE
:10305D00FFE5642FFF50010E900025EEF0A3EFF079
:10306D00900098E0048E048F05FF12686F8D6480C8
:10307D00037564329000E4E07006756E03022C7ADD
:10308D0075BB130233F39000E4E0604A7E017F00CC
:10309D00E5BE12687FE5BD2FFF50010E8E598F5A88
:1030AD0074041200398F659000E6E08565F0A4FD8B
:1030BD00ACF07464FF12686F8D659000E5E0856576
:1030CD00F0A4FFAEF074FF8E048F05FF12686FED54
:1030DD0090007FF08003756500900092E07006759A
:1030ED006E04022C7A75BB170233F3900092E0B494
:1030FD000102800302318C7E017F00E5BE12687FE4
:10310D00E5BD2FFF50010E8E598F5A9007DEE060FE
:10311D00199007DEE0149062F912008CE493FC74B0
:10312D000193FDEDC39FEC9E400280069007DEE00B
:10313D0014F09007DEE0C394B3501DAE59AF5A9012
:10314D0007DEE0049062F912008CE493FC740193A5
:10315D00FDEFC39DEE9C400280069007DEE004F07B
:10316D009007DEE0FE9000B8E08E0088F0A4FFAE80
:10317D00F074648E048F05FF12686F8D6680037581
:10318D006600900093E07006756E05022C7A75BB93
:10319D00160233F3900093E0B4010280030232353E
:1031AD007E017F00E5BE12687FE5BD2FFF50010E49
:1031BD008E598F5A9007DFE060199007DFE0149069
:1031CD00646312008CE493FC740193FDEDC39FECDA
:1031DD009E400280069007DFE014F09007DFE0C309
:1031ED0094B3501DAE59AF5A9007DFE0049064635D
:1031FD0012008CE493FC740193FDEFC39DEE9C4093
:10320D000280069007DFE004F09007DFE0FE9000FB
:10321D00BEE08E0088F0A4FFAEF074648E048F05BE
:10322D00FF12686F8D67800375670075BB1F0233D2
:10323D00F37E017F00E5BE12687FE5BD2FFF5001D3
:10324D000E8E598F5A740912687F74E68E048F059D
:10325D00FF12686F8D6990009AE07006756E070217
:10326D002C7A75BB150233F390009AE0700302338C
:10327D008F7E017F00E5BE12687FE5BD2FFF5001F7
:10328D000E8E598F5A74041200398F6890009AE08F
:10329D00B401159000EEE08568F0A4FFAEF0740760
:1032AD00120039EF9007D3F090009AE0B402159018
:1032BD0000EEE08568F0A4FFAEF07407120039EF60
:1032CD009007D2F090009AE0B40302800302338D90
:1032DD009000DBE070389000EEE0601CE568C39470
:1032ED00195002D22AE568D394644002C22A900094
:1032FD00BAE09007D6F08014E568C394195002D255
:10330D0039E568D394324002C239C22A80639000F5
:10331D00BAE070349000EEE08568F0A4FFAEF07472
:10332D00FF8E048F05FF12686FED9007D6F0AE513A
:10333D00AF52741EBE0006D39F4002D22AE560D361
:10334D0094E54002C22A8029E568C3940A500DAE67
:10335D0051AF52741EBE0004D39F50028002D22A78
:10336D00E560D394E54002C22A9000BAE09007D6FA
:10337D00F09007D6E0C39405500674059007D6F07B
:10338D0080037568009000F1E07006756E08022CE0
:10339D007A75BB1480509000F1E060397E017F009A
:1033AD00E5BE12687FE5BD2FFF50010E8E598F5A75
:1033BD00EFD39421EE940E4005756AFF8015AE593A
:1033CD00AF5A741012687F74E38E048F05FF126874
:1033DD006F8D6A8003756A00900095E0600575BB7E
:0633ED001A800375BB18F5
:10359F00022C83022E3D022FDE0230930230F802FE
:0B35AF0031A102323E0232750233A34C
:0533F300056ED2EC2282
:0968B1002582F5825002058322C4
:0F008C0025E050020583258250020583F582226C
:10684E00EF2F500205832582F582E5833E2EF583D8
:01685E002217
:1068C300CFC39FFF50011E22C3EF9DFFEE9CFE220C
:0868D3000806B60002180622B7
:0D688D00A3E004F07006120049E004F022C0
:0E003900048007C3CE13CECF13CFD5E0F6223E
:10676D00BC000FBE0008ED8FF084FFADF022E4FEFB
:10677D00FF22BE000DEF60FE54F0606F20E70302B4
:10678D006823EAC0E0EBC0E078017A0075F001EE15
:10679D0020E710EF25E0FFEE33FE0AC5F023C5F02C
:1067AD0030E7F0EA5407F9096A7A007B00600108C6
:1067BD00C3EC9E40167004ED9F4010ED9FFDEC9EC6
:1067CD00FCE5F0CA4ACA03F5F08005E5F003F5F0E3
:1067DD00C3EE13FEEF13FFD9D77908CACBCAD8D0B1
:1067ED00EAFEEBFFD0E0FBD0E0FA22EC8FF084FC68
:1067FD00ED54F045F0C48FF084FEEDC454F045F037
:10680D00C48FF084FDEEC4FE54F02DFFEE540F3C0A
:10681D00FEADF07C0022790078008FF0EC7E082030
:10682D00E70DC3CD33CD33C933C9C833C8DEF084CA
:10683D0049F9E5F08FF0BE00E6FD7C00E9FFE8FECA
:01684D002228
:0E687F00F88FF0A4FFE5F0CE88F0A42EFE22E4
:10000300EF8DF0A4F9A8F0EF8CF0A428F8EE8DF0B2
:06001300A428FEE9FF2213
:10685F00600D782B026869007830D8FED5E0F822F9
:10686F00EEC0E07E0012676DEFFDEEFCD0E0FE2281
:0C689A00EEC0E07E0012676DD0E0FE2230
:03001B0002001EC2
:0300530002005652
:03009B00020071EF
:030000000268BAD9
:0968BA0075817475D000024030B4
:0B68A600E5822FF582E5833EF583229A
:0A0049000582D5820215831582227C
:10001E00C0E0C0F0C083C082C0D075D000123F5E79
:0B002E00D0D0D082D083D0F0D0E032E0
:10005600C0E0C0F0C083C082C0D075D000123F613E
:10006600D0D0D082D083D0F0D0E032C0E0C0F0C093
:1000760083C082C0D075D000123FE3D0D0D082D0EA
:0600860083D0F0D0E0324F
:00000001FF
